:1000000000800020BD010000993D0000993D0000E6
:10001000993D0000993D0000993D0000653D0000BC
:10002000653D0000653D0000653D0000993D000014
:10003000993D0000653D0000993D0000553D0000E0
:10004000993D0000993D0000993D0000993D000058
:10005000993D0000993D0000993D0000993D000048
:10006000993D0000993D0000993D0000993D000038
:10007000993D0000993D0000993D0000993D000028
:10008000993D0000993D0000993D0000993D000018
:10009000993D0000993D0000993D0000993D000008
:1000A000C1380000993D0000993D0000993D0000D5
:1000B000993D0000993D0000993D0000993D0000E8
:1000C000993D0000993D0000993D0000993D0000D8
:1000D000993D0000993D0000993D0000993D0000C8
:1000E000993D0000993D0000993D0000993D0000B8
:1000F000993D0000CD580000993D0000495D000089
:10010000993D0000F9600000993D0000993D000014
:10011000993D0000993D0000993D0000993D000087
:10012000993D0000993D0000993D0000993D000077
:10013000993D0000993D0000993D0000993D000067
:10014000993D0000993D0000993D0000993D000057
:10015000993D0000993D0000993D0000993D000047
:10016000993D000095440000993D0000993D000034
:10017000993D0000993D0000993D0000993D000027
:10018000993D0000993D0000993D0000993D000017
:10019000993D0000993D0000993D0000193F000085
:1001A000693F0000F13F0000AD4000003141000018
:1001B000993D0000993D00001D500000544B4CF249
:1001C000205210B51A804DF628121A8000BF00BFC9
:1001D00003F0E6FD4F4B4FF010621A604E4A9A60F2
:1001E0004E4ADA604E4B1A6812F4807204D14D49BF
:1001F0000A604FF4A8521A604B4B1A7802F00802BA
:10020000D2B21AB11A7842F008021A70474B484825
:10021000484C2A221A700023474A02E01959995083
:10022000043399188142F9D3444B454A002101E037
:1002300043F8041B9342FBD34249434800231A5816
:100240005A500433B3F5DE7FF9D1404B404A802148
:1002500003F8011B9342FBD13A4A3E4B1A603E4BD6
:100260000A221A703D4B24221A70A02203F8012C96
:100270003B4A137803F00203DBB2002BF9D0384A73
:10028000137803F01003DBB2002BF9D1344A137852
:1002900003F00C03082BFAD1324B03221A704022D0
:1002A0005A702F4A137803F02003DBB2002BF9D0E9
:1002B0002B4A137803F04003DBB2002BF9D02A4B12
:1002C0002A4A1A6002225A60294B20221A70244AB4
:1002D000137803F00C030C2BFAD1264A264B1A6034
:1002E000264B274A1A60072243F8042C62B603F013
:1002F000C3FF0C4B1B68DC0702D5224803F030FF1C
:1003000008F02CFA03F052FD04F034FFFEE700BFC2
:100310000E20054030800440823F04000100002B85
:1003200010D0034014D0034002D0074000E0074043
:100330005895FF1FFCA70000608FFF1F5895FF1FF7
:10034000DCA9FF1F008AFF1F0000000000E400E09E
:100350005FE400E008ED00E0005006400140064088
:10036000064006400440064044800440000003016B
:1003700000400640C01005000480044014E000E086
:10038000FF7601008E0AFB54FFFFFFFFFFFFFFFF18
:10039000FFFFFFFFFFFFFFFFFFFFFFFFFFFFFFFF6D
:1003A000FFFFFFFFFFFFFFFFFFFFFFFFFFFFFFFF5D
:1003B000FFFFFFFFFFFFFFFFFFFFFFFFFFFFFFFF4D
:1003C000FFFFFFFFFFFFFFFFFFFFFFFFFFFFFFFF3D
:1003D000FFFFFFFFFFFFFFFFFFFFFFFFFFFFFFFF2D
:1003E000FFFFFFFFFFFFFFFFFFFFFFFFFFFFFFFF1D
:1003F000FFFFFFFFFFFFFFFFFFFFFFFFFFFFFFFF0D
:10040000FFFFFFFFFFFFFFFFFFFFFFFFFEFFFFFFFD
:1004100008B549F25850074BC1F6FF701B1A062B5E
:1004200000D808BD40F20003C0F20003002BF8D052
:100430009847F6E75B95FF1F08B549F2585049F217
:100440005853C1F6FF70C1F6FF731B1A9B1003EBE4
:10045000D373591000D108BD40F20002C0F200026F
:10046000002AF8D09047F6E710B549F25854C1F683
:10047000FF74237873B9FFF7CBFF40F20003C0F29B
:1004800000032BB14AF2FC70C0F20000AFF3008011
:100490000123237010BD00BF08B540F20003C0F275
:1004A00000034BB14AF2FC7049F25C51C0F200000B
:1004B000C1F6FF71AFF3008049F25850C1F6FF70EA
:1004C00003682BB140F20003C0F2000303B1984768
:1004D000BDE80840FFF7B0BF044A10B5044640F835
:1004E0001C2B01F02FFD204610BD00BF58A20000BC
:1004F00038B5054CA4F517652046103C04F0CCFE39
:10050000AC42F9D138BD00BFE0A2FF1F38B50446A8
:1005100008460D4603F074FC236802465B682046DB
:100520002946984738BD08B5FFF7F0FF08BD38B534
:100530000446FFF7EBFF0546204604F035FE281879
:1005400038BD38B50A220023044604F03BFE0546B8
:10055000204604F029FE281838BD38B5044604F0BA
:1005600069FE0546204604F01FFE281838BDFFFF2F
:10057000034B82B01B680193019B036002B070477C
:10058000B4A6FF1F044B00681B6882B00193019B57
:10059000181A02B0704700BFB4A6FF1F044B82B008
:1005A0001B680193019B591A016002B0704700BF9C
:1005B000B4A6FF1F0F4B4172036000230261037258
:1005C000C360194603E0026942F823100133427AFE
:1005D0009342F8DB084A136813B9106004E013462D
:1005E0005A69002AFBD15861002343618380C3808C
:1005F000704700BF189E0000ACA7FF1F0B79037166
:100600008B6883600B7B30B5037300F10D0201F141
:100610000D0301F1190453F8045BA34242F8045B93
:10062000F9D11B781370CB69C36130BD30B5254B50
:1006300025498DB004AC4FF080421A602046234A11
:10064000012301F0F9FD21462148FFF7D7FF20469D
:1006500001F078FC1E4801F093FE002520461C495D
:10066000012201F04FFE204601F0B1FCF8B1204616
:1006700001F06EFC0146684604F04FFE204601F092
:1006800069FC40B1684604F02BFF70B96846114917
:1006900004F0C4FE48B9204601F08DFC684604F021
:1006A000FBFD204601F04EFCD8E70135F3E720467C
:1006B00001F048FC084B4FF080421A6028460DB00C
:1006C00030BD00BF88E100E04CA3FF1F549E000036
:1006D0007895FF1F569E000008E100E070B5444B7E
:1006E000444996B04FF080421A60044602A804F0D4
:1006F00014FE214602A804F079FE3E4902A804F047
:100700005AFE02A869460422002304F0D1FE3A48AA
:10071000694601F0E3FD054620B938493848FFF73E
:1007200006FF5EE00EAC6A4601232046324901F026
:1007300083FD21463348FFF761FF204601F002FCAC
:10074000304801F01DFE002520462E49012201F00F
:10075000D9FD204601F03BFC002833D0204601F0B3
:10076000F7FB014606A804F0D8FD06A8264904F0C8
:1007700089FEE8B125490AA804F0CFFD06A80AA918
:1007800004F077FE30BB952DCCBF0026012622E079
:10079000204601F0DDFB01461D4800EB051004F08A
:1007A000E2FD204601F0F0FB1A4B43F8250001352D
:1007B000204601F000FC06A804F06EFD204601F082
:1007C000C1FBC1E7204601F0BDFB134B4FF0804257
:1007D0001A6006E000260AA804F05EFD002ED7D1BC
:1007E000E6E702A804F058FD284616B070BD00BF29
:1007F00088E100E0549E00004CA3FF1F589E0000BB
:10080000DCA7FF1F7895FF1F2499FF1F6C9E000037
:100810008099FF1FE495FF1F08E100E070B5114CBF
:100820008AB006460D4601A8214604F076FD314601
:1008300001A804F0DBFD214601A804F0BCFD0A4933
:1008400001A801EB051104F0B1FD01A805A91222D0
:10085000002304F02DFE01A804F01EFD05A80AB037
:1008600070BD00BF549E00008099FF1F08B54FF473
:10087000FA7003F0EBFC024A024B1A6008BD00BF9D
:100880000400FA050CED00E010B50446C4F3C00105
:10089000062003F075FC0520C4F3800103F070FC12
:1008A0000420C4F3400103F06BFC032004F00101B9
:1008B00003F066FC0B20C4F30011BDE8104003F008
:1008C0005FBCFFFFFFFFFFFF38B572B6384A137FEA
:1008D0000BB10021117762B6002B62D000213548A0
:1008E000FFF75CFE72B6324BB3F91E20B3F920005D
:1008F000801A47F6FF72DA834FF400421A8462B618
:1009000007F092F828A3D3E9002307F01DFA07F0B7
:10091000B3FB4FF0814107F0FFFB0021044607F0D5
:10092000ADFD38B1204607F091F80022224B06F0C9
:100930002FFF06E0204607F089F800221E4B06F044
:1009400025FF07F071FB07F06FF804460D462246BD
:100950002B4600204FF0804105F0B2FD002200231D
:1009600007F04EFB58B122462B4600204FF0804145
:1009700005F0A6FD0022104B06F00AFF0AE0224611
:100980002B4600204FF0804105F09AFD00220A4BD3
:1009900006F0FCFE07F048FB0138BDE83840FFF7E1
:1009A00073BF38BDAFF3008000000000E0FFEF40F0
:1009B0004498FF1F7C99FF1F0000E03FAFF30080C9
:1009C00008B504F08DFD431E5842584108BDFFFF95
:1009D00030B50C4685B04B49054604F01FFD58B1B3
:1009E0002146684604F0B4FC6846FFF7E9FF464B31
:1009F0001870684604F050FC2846444904F00EFD87
:100A000020B1204604F06CFD414B18602846414956
:100A100004F004FD58B12146684604F099FC68468C
:100A2000FFF7CEFF3C4B1870684604F035FC2846B3
:100A30003A4904F0F3FC20B1204604F051FD384B54
:100A400018602846374904F0E9FC58B12146684649
:100A500004F07EFC6846FFF7B3FF334B187068461E
:100A600004F01AFC2846314904F0D8FC58B121465C
:100A7000684604F06DFC6846FFF7A2FF2C4B187027
:100A8000684604F009FC28462A4904F0C7FC58B11E
:100A90002146684604F05CFC6846FFF791FF264B50
:100AA0001870684604F0F8FB2846244904F0B6FCA8
:100AB00058B12146684604F04BFC6846FFF780FFBA
:100AC0001F4B1870684604F0E7FB28461D4904F0E8
:100AD000A5FC20B1204604F003FD1B4B18602846FE
:100AE0001A4904F09BFC58B12146684604F030FCDA
:100AF0006846FFF765FF164B1870684604F0CCFB9C
:100B000005B030BDF49E00001499FF1FF99E00004F
:100B1000708FFF1F019F0000788FFF1F0B9F000049
:100B20006C8FFF1F159F0000848FFF1F269F000002
:100B3000948FFF1F369F00000899FF1F489F0000F9
:100B4000C898FF1F599F0000888FFF1F689F0000F3
:100B50008C8FFF1F30B59DB00021684604F0DDFB8F
:100B6000002104A804F0D9FB3B4A3C49012314A806
:100B700001F062FB14A93A48FFF740FD14A801F008
:100B8000E1F937486C4601F022FA002857D06C464C
:100B9000334801F0FDF900284DD00EE0694608A861
:100BA00004F0D6FB294608A804F032FC014668464A
:100BB00004F0C6FB08A804F06FFB294801F06DF9AA
:100BC000C5B23D2DEAD1264801F067F9C5B22FE044
:100BD00004A908A804F0BCFB294608A804F018FCE6
:100BE000014604A804F0ACFB08A804F055FB1C481F
:100BF00001F053F9C5B20A2D1AD169460CA804F0C8
:100C0000A7FB04A910A804F0A3FB10A90CA8FFF7E8
:100C1000DFFE10A804F040FB0CA804F03DFB684682
:100C2000104904F0A0FB04A80E4904F09CFBAFE7B8
:100C30000A2DADD0CCE70A4801F0BDF903E00A481F
:100C40000A49FFF774FC04A804F026FB684604F088
:100C500023FB1DB030BD00BF7E9F00004CA3FF1FD3
:100C6000BC95FF1F15A00000DCA7FF1F709F0000B0
:100C700030B53A4D3A4C89B02146284601F038FB50
:100C80002246384C13236846294601F0D5FA6946B6
:100C90002046FFF7B3FC684601F054F9204632497C
:100CA000FFF741FC314B20461978FFF74AFC2046FC
:100CB0002F49FFF738FC2F4B20461968FFF74DFCF2
:100CC00020462D49FFF72FFC2C4B20461978FFF7C3
:100CD00038FC20462A49FFF726FC2A4B2046196893
:100CE000FFF73BFC20462849FFF71DFC274B204619
:100CF0001978FFF726FC20462549FFF714FC254B01
:100D000020461978FFF71DFC20462349FFF70BFC0E
:100D1000224B20461978FFF714FC20462049FFF7A4
:100D200002FC204B20461978FFF70BFC20461E4999
:100D3000FFF7F9FB1D4B20461968FFF70EFC204614
:100D40001B49FFF7F0FB1B4B20461978FFF7F9FB17
:100D5000204601F030F909B030BD00BF4CA3FF1FA1
:100D60007E9F0000BC95FF1F879E00001499FF1F07
:100D70008D9E0000708FFF1F969E0000788FFF1FD2
:100D8000A19E00006C8FFF1FAC9E0000848FFF1F90
:100D9000BE9E0000948FFF1FCF9E00000899FF1F8A
:100DA000E29E0000C898FF1F8B9F0000888FFF1FE6
:100DB0009B9F00008C8FFF1F30B5022089B000215F
:100DC00003F00AFA0820002103F006FA09200121A5
:100DD00003F002FA0B20012103F0FEF906200121A5
:100DE00003F0FAF90520012103F0F6F904200121AE
:100DF00003F0F2F90121032003F0EEF9404B1868EB
:100E0000FFF742FD4FF47A7003F020FA3D480521C8
:100E100003F0FEFF3C4B3D481A780A2142F00502E0
:100E20001A7001F06DF918B3394A38490123684640
:100E300001F002FA69463748FFF7E0FB684601F027
:100E400081F83248344901F049FAC8B91BE00F2053
:100E5000FFF71AFD642003F0F9F92846FFF714FDA7
:100E60000134642003F0F2F9062C01DDFFF7FEFCEB
:100E700026480A2101F044F905460028E7D0D3E7C7
:100E8000FFF768FE01E0FFF7F3FEFFF7CFFB234C0F
:100E900001462060224804F0CDF922492048FFF79E
:100EA00046FB0021204800F0D3FB2368013B984219
:100EB00005DA134B18601D4B01221A7004E0002163
:100EC00019480A4600F0C7FB0D4C19491448FFF7B2
:100ED0002AFB21681248FFF740FB2068FFF7FEFB62
:100EE000144B014618600E4804F0A4F912490C484E
:100EF000FFF719FB21680A48FFF72FFB09B030BD47
:100F0000DC95FF1F0082FF1FD6A7FF1F4CA3FF1F0A
:100F1000549E00007895FF1F7E9F00004499FF1F9C
:100F2000DCA7FF1FA49F0000F4A2FF1F648FFF1F18
:100F3000B19F0000CC98FF1FBB9F00002DE9F04F30
:100F4000002495B0264625462746A146DFF8B882FC
:100F500010E0172002F014FE8144142002F010FE6D
:100F60003F18152002F00CFE2D18162002F008FE86
:100F700001343618D8F800309C42EADB95FBF3F5D3
:100F800096FBF3F699FBF3F997FBF3F7834B844A4F
:100F9000D3F800A0834B12681B6802920393824B24
:100FA0001B68EB1A83EAE372A2EBE3727F4B0492B5
:100FB000D3F800B07E4B1B68F31A83EAE372A2EB0E
:100FC000E37209EB070040F2FF339842A8BF1846CE
:100FD000784B05921B68002100934FF480620B460A
:100FE00020EAE07004F04EF9DFF820E28046BEE827
:100FF0000F0007AC0FC4BEE80F000FC4BEE80F001F
:101000000FC4DEF800300021236005EB060C0D2331
:1010100040F2FF30844538BF60464FF48062009351
:101020000B4604F02FF90446634800F077FE14AA3B
:1010300002EB8404614A54F8343CB0FBF3F0604B9B
:1010400010601B6898451CD0029AC2EB0903002B64
:10105000B8BF5B42534540F395805A4BC3F80080BC
:10106000594B1A78594B1A704D4BC3F8009089E0D0
:10107000544BC3F80080564B1A78544B1A70494BA6
:101080001F60049A53485A45C4BF474B1D60059BD7
:101090005B45C4BF464B1E6000F016FB20B14D48B7
:1010A00000F0F4FA4C4B18704C48FFF76BFA04460A
:1010B000082003F085F804FB00F14848FFF76EFABA
:1010C0004648FFF75FFAB0F5C87F64D9444C454AFB
:1010D0002368126801339A42236001DC00232360F5
:1010E00041494248334DFFF71EFA21683F48FFF758
:1010F00034FA2068FFF7F2FA0028286003DC3B4846
:101100003B49FFF714FA296838482E4C04F092F84E
:1011100038493648FFF707FA314B34481968FFF76A
:101120001CFA35493148FFF7FEF930482168FFF7CE
:1011300014FA2B682268934201DC013B2360236888
:10114000002B02DA1F4B00221A602C492748FFF7B8
:10115000EAF91C4B25481968FFF7FFF91B4B1F489C
:10116000012200211A70FFF719FA00212448FFF725
:1011700015FA1B4B23481A78002115B0BDE8F04F33
:1011800000F069BA039ABB1A002BB8BF5B42534503
:101190003FF76EAF75E715B0BDE8F08F908FFF1F7A
:1011A0009895FF1FF0A2FF1F7495FF1F808FFF1FF0
:1011B0009C95FF1FCC98FF1F8098FF1F988FFF1FE3
:1011C0001C99FF1F4C99FF1F848FFF1F648FFF1F07
:1011D000948FFF1F3499FF1F6898FF1F6C98FF1FA3
:1011E000DC95FF1F4499FF1FD19F0000DCA7FF1F64
:1011F000E49F0000BB9F0000F39F00000CA00000D4
:101200004098FF1FF4A2FF1F748FFF1F209E000055
:1012100038B57B487B4DFFF7B5F90A22014600231C
:10122000794803F0CFFF784803F0BEFF95F84440BB
:1012300024B9764B1B78002B40F0C480714B1B7E89
:101240000BB1FFF713FB724B1B781BB9714B1B786B
:10125000002B5ED0704B1B789BB1704C704823689C
:1012600040F2B912534305330A22B3FBF2F34FF0B5
:10127000FF31B1FBF3F1002200F0C4FA206802F064
:10128000E5FF684C684B21681868FFF7C7FA674BA1
:1012900022681860664B674C1A605E4B1B7833B946
:1012A0005A4B1B781BB1574800F040FD2060226864
:1012B0005E4B5448196822F00F02226000F0DEFCF9
:1012C000554B1B7883B1554B55481B6840F2B912FA
:1012D000534305330A22B3FBF2F34FF0FF31B1FB66
:1012E000F3F1012200F08EFA4F4B1868FFF7CCFAA9
:1012F000474B434800241C70464B21461C70FFF7A7
:101300004DF921464C48FFF749F94C482146FFF773
:1013100045F94B48FFF736F94A4B1B68984205D30D
:10132000FFF70CFE46480021FFF738F94648FFF763
:1013300029F9464B1B68984203D943480021FFF71F
:101340002DF9394B2E481B680F2B06DCFFF71AF9D5
:1013500009288CBF0021012105E0FFF713F90A28B5
:1013600094BF002101210B2002F00AFF3848FFF74B
:1013700009F953280AD93748FFF704F9364B1B6897
:10138000984203D9354B1B78002B35D12B48FFF7FA
:10139000F9F8334B196888422CBF0021012109203C
:1013A00002F0EEFE2448FFF7EDF82E4B1B68984242
:1013B00025D900212048FFF7F1F800211F48FFF749
:1013C000EDF838BD184B1868194B1968FFF726FA65
:1013D000164B224618600146284600F04FFC214675
:1013E0000748FFF7DBF821461348FFF7D7F82146F7
:1013F0001248FFF7D3F821E7FFF766FAC6E738BDD2
:10140000E098FF1F8098FF1FDCA7FF1F8C8FFF1F36
:10141000648FFF1F6898FF1F1499FF1F708FFF1FB5
:101420005499FF1F4C99FF1FDC95FF1FE498FF1F85
:101430001C99FF1FE095FF1F0C99FF1F1099FF1FBC
:101440004899FF1F9C8FFF1F5099FF1F688FFF1F38
:101450007C99FF1F4098FF1F6C8FFF1F788FFF1F25
:101460007C8FFF1F988FFF1F2DE9FF415648574D76
:10147000574F584EDFF8D48100F056FD5649574A71
:10148000514807F04DF900210A462846FFF792F827
:10149000534B2846002440F81C3B00F045FD2846ED
:1014A00000F0C8FB28464F494C4A07F039F90121A2
:1014B00007F124023846FFF77DF84B4B01213B60D2
:1014C00006F118024FF0FF333046BB61FFF772F8A8
:1014D000464B336047F6FF7308F118020121F3838E
:1014E00040464FF400433384FFF764F8404B4046D6
:1014F000C8F8003000F052FA3E4880E8A0000472BC
:101500004472C46003F05DFD3B4880E880010472D2
:101510004472C46003F055FD384880E860000472EE
:101520004472C46003F04DFD35493648364D03F032
:10153000F4FE3649294A334807F0F2F8344800F0FF
:10154000F3FC33482449254A07F0EAF8281900211A
:10155000103403F0E2FEB4F5176FF7D100202D49E7
:101560001E4A07F0DDF8082114222B4800F07AF813
:1015700002211422294800F075F82948FEF7F8FFE7
:101580002848FEF7F5FF2848FEF7F2FF274B2848CA
:101590001A6801920199274A11601A680292029909
:1015A0001B68254A03931160244B039A1A60FEF7C7
:1015B000DFFF2348FEF7DCFF2248FEF7D9FF224871
:1015C000FEF7D6FFBDE8FF81BC95FF1F8098FF1F87
:1015D0005499FF1F4498FF1F451F0000608FFF1F95
:1015E00058A20000D904000038A2000028A2000080
:1015F00048A200007098FF1FE898FF1FF898FF1F8F
:1016000016A000002499FF1F8099FF1F9952000027
:101610007895FF1FF10400003499FF1FD098FF1F39
:101620002099FF1F1899FF1F5099FF1FB4A6FF1F95
:101630004098FF1FE098FF1F6C98FF1F4899FF1FFD
:101640007C99FF1F1099FF1F0C99FF1FA095FF1F8A
:10165000084602F051BB0846114602F061BB02F099
:101660000FBBFFFF37B500238360074B42601B6849
:101670000193019B0446036008460D4602F0A0FD5D
:101680006573207320463EBDB4A6FF1F007B7047E4
:1016900013B50446407B02F093FD237B834201D1C6
:1016A00000200EE0074B1A68009200992268891A00
:1016B00062689142F4D31B6820730193019B01205F
:1016C00023601CBDB4A6FF1F37B50446FFF7E0FF3B
:1016D00010B10023A3600EE0A26872B1084B196834
:1016E0000091009D2168691A914206D31B68A06091
:1016F0000193019B2360012000E00020A0733EBD08
:10170000B4A6FF1F70B50021044603F02CFCC0B145
:10171000B4F91E20B4F92030811C00F5817631F92E
:10172000025BAA42A8BF2A46AB42B8BF2B46B142D1
:10173000F5D323840123E2832377BDE8704003F0CF
:10174000DDBB70BD2DE9F047846905462CB9214603
:1017500003F009FC002851D04CE00021631C0BD1A0
:1017600003F001FC0446002848D028462146002208
:1017700003F0E4FB20463DE003F002FC06460028AF
:101780003CD0EA6995F820101D4800234FEA146CFC
:10179000C4F30F2E30F91CA00CF1010CF71830F92E
:1017A0001CC0B7F90280CEF580390EFB0CFC0AFB99
:1017B00009CE4FEA2E4E0EFB08FE4FEAEE3EA7F88A
:1017C00002E021B1E743BA4205D2A41807E0A242E1
:1017D00004D2A41A03E04FF0FF3400E00C460233B9
:1017E000B3F5807FD2D12846AC613146002203F0A8
:1017F000A5FB3046BDE8F04703F080BBBDE8F087AD
:101800001AA0000072B683690BB9012303E001330B
:1018100002D16FF001038361C16180F8202062B6BC
:101820007047FFFF2DE9F041DFF860C0154E164FFD
:10183000002A0CBF4FF064524FF06052002434F87D
:10184000078056F814509CFBF8F8414504D303F088
:101850000801C9B221B905E002342E2CEFD1F6E718
:1018600042F0806203F00403DBB23BB125F4704325
:1018700005F4704542F0007243EA15152A430260F0
:10188000BDE8F08194A2000064A20000006CDC02BC
:1018900010B50446FFF7C6FF204610BD10B504463C
:1018A00003F04EFC204610BD02480349034A06F0EF
:1018B00037BF00BFF8A2FF1F9D180000608FFF1FF9
:1018C00002480349034A06F02BBF00BF00A3FF1FD5
:1018D0009D180000608FFF1F10B5194B1A68116822
:1018E0001A79184B1A70184A9142184928BF184B98
:1018F00008683CBF134603F5807298B1014631F980
:10190000024F04F5FF447F34241123F8024B934225
:10191000F5D303F0F3FA0F4B0C491A680A60002262
:101920001A6005E040F2FF7123F8021B9342FBD3DB
:10193000094B1B781BB1094B4FF080421A6010BD58
:101940000CA3FF1F1F8000400A88FF1F18A3FF1F62
:101950000A87FF1F08A3FF1F14A3FF1F08E200E070
:1019600010B5002103F0FFFA034690B172B60949A1
:10197000086808B90B6003E0074A146814B91360DB
:1019800062B610BD0C60136062B6BDE8104003F093
:10199000B5BA10BD18A3FF1F08A3FF1F38B54B48E9
:1019A0004B4D012103F074FB4A4B1A6842F48052FC
:1019B0001A60494B80221A7000242C8008340120C0
:1019C000A4B202F043FCB4F5006FF6D1434B1B68A0
:1019D0005B0264D5424B1A6848F6A273134048F67E
:1019E000A27293425BD13F4B1A6840F23F439A4246
:1019F00055D13D4B1B68012B51D13C4B1A6840F22D
:101A000001139A424BD1314D39492B681A6819603C
:101A10000221197119726FF0010159734FF0FF31F2
:101A20009973D97319692A494FF48070196100229A
:101A3000D98AD88211465A715A729A72DA721A7316
:101A40001A755A751A765A769A76DA76DA8BD883B8
:101A50009A8B012406229A839C71DC712B7903F105
:101A6000804303F50433B02219701A7003F0C0FAF2
:101A7000204B214A18702B792048137003F1100174
:101A80001F4A42F821005A11920002F1604202F509
:101A9000614203F01F0304FA03F4146038BD0F4BD6
:101AA0001A6842F480021A600F4B01221A6040F259
:101AB0003F4243F8082C48F6A37243F80C2C114A15
:101AC00043F80C2C40F201125A609CE70CA3FF1F54
:101AD00000C00C402C80044021C00C403C800440DD
:101AE00000600340046003400C600340106003404A
:101AF0000A87FF1F14A3FF1F1B800040D918000096
:101B0000008AFF1FA28F010002480349034A06F022
:101B100007BE00BF0CA3FF1F9D180000608FFF1FB2
:101B200002480349034A06F0FBBD00BF1CA3FF1F88
:101B30009D180000608FFF1F02480349034A06F00A
:101B4000EFBD00BF24A3FF1F9D180000608FFF1F83
:101B5000F8B590F844300446002B64D003F086F9C1
:101B6000054600285FD004F11C06304600F010FA4C
:101B700000283ED0A91C30464FF4807200F0F2F9E4
:101B8000B0F5807F074621D9274D28492B680322CD
:101B90005B68284698470A2200233946284603F006
:101BA00011FB284603F000FB304600F004FA204AFF
:101BB0001388002B2FD0013B9BB21380002B2AD01F
:101BC000002384F8443001232376F8BD236CC31826
:101BD000236400232376470803E005EB470201371F
:101BE0005380802FF9D120462946002203F0A6F920
:101BF0000CE0304600F0DFF90D4A13887BB1013B61
:101C00009BB213805BB1002384F844302846BDE8C2
:101C1000F84003F073B95E2000F0F0F8D0E75E20E2
:101C200000F0ECF8EFE7F8BDDCA7FF1F60A20000B2
:101C30002CA3FF1F002380F84430C3630364704764
:101C400008B572B690F8443073B1002380F8443080
:101C500062B61C3000F0AFF9074A138833B1013B7C
:101C60009BB2138013B108BD62B608BD5E20BDE80B
:101C7000084000F0C3B800BF2CA3FF1FF0B589B027
:101C8000154604460F46FFF7DBFF5E2000F09CF888
:101C9000204B1A8801321A8072B61F493A46012336
:101CA000684600F0C9FA9DF8043084F82030029BA1
:101CB00063629DF80C3084F828300DF10D0304F1B7
:101CC0001C0604F1290203F10C0153F8040B8B42AA
:101CD00042F8040BF9D11B781370079B6846A36385
:101CE00000F030F962B6304600F071F978B1304654
:101CF00000F04AF90346B5FBF0F1E06303FB115134
:101D0000304600F035F90120256484F8440009B01C
:101D1000F0BD00BF2CA3FF1F4CA3FF1FC26B024BE3
:101D2000A2FB032318467047C8BDE602006C70474B
:101D3000184B19491A6842F480521A60174B184A16
:101D40001A60184A116001F180415160164A1A6008
:101D5000164B1B78DA0755BF154A164A4FF4107117
:101D60004FF40071116003F00201C9B24FF4007228
:101D700009B9114900E0114903F00403DBB20A601C
:101D80001BB94FF410720E4B02E00E4B4FF4007271
:101D90001A6070473C8004400110003800C00240C7
:101DA00001401F000CC0024000001F80D6A7FF1F8B
:101DB00018B0044008C004401CB004400CC00440EB
:101DC00014B0044004C004405E2830B511D8094A5C
:101DD00043091478012101FA03F52C431470064AD3
:101DE00000F01F0052F8234001FA00F10C4342F8C2
:101DF000234030BD48A3FF1F30A3FF1F5E2810B54E
:101E000014D843090A4A00F01F0052F82340012168
:101E100001FA00F024EA000042F8230030B9054A34
:101E2000107801FA03F320EA0303137010BD00BF1A
:101E300030A3FF1F48A3FF1F13B502AB026803F8CE
:101E4000011D546819460122A0471CBDC06908B194
:101E500001F026B8704738B50446C069002510B9AE
:101E60000123237138BD0571E06992B201F09AF93E
:101E7000E3691B7913B101232371284638BD07B5E7
:101E800001220DF1070100F0FBFE01280CBF9DF8B7
:101E900007004FF6FF7000B20EBDC06908B510B163
:101EA000FFF7EDFF08BD4FF0FF3008BD38B5054620
:101EB000C06950B1FFF7E3FF431C044606D0E86950
:101EC000C168013900F0B8FF00E00446204638BD83
:101ED000F8B504464FF47A73A360124B00202071CA
:101EE0002073236024200D46174606F063FCE06152
:101EF000A8B12B4603F120020546186859682E4602
:101F000003C6083393423546F7D118683946306026
:101F10000C2204F10D0007F00BFD00236376204630
:101F2000F8BD00BFF8A200004FF47A718160044947
:101F30000022027102730160C2614273704700BFE8
:101F4000F8A20000014B0360704700BFF8A2000038
:101F50000D307047C06920B18079012894BF0020FE
:101F600001207047C06908B508B100F089FE08BDBE
:101F7000C06908B100F060BF7047C3690BB1D86891
:101F800070474FF0FF307047C06900B180697047FB
:101F900038B5C369044663B1FFF7F6FF054620462E
:101FA000FFF7EBFF47F6FF73281A984228BF184641
:101FB00038BD184638BD10B50446C06930B100F0D0
:101FC0009BFFE06906F0FEFB0023E36110BDC069E2
:101FD00018B18079003018BF0120704710B50A464B
:101FE0008AB00A49044600238DF8083001918DF823
:101FF0000A30214601A8012301F034F8044610B14B
:1020000001A800F079FF20460AB010BD28A3000007
:102010000AB101F0AFB80120704770B50B68C45C1D
:102020002F2C08BF0133C6180024355D2F2D08D092
:102030006DB906E001330B60C05C003018BF0120B1
:1020400070BD00251555C25C2F2AF4D1F2E7155555
:10205000013401330C2CF4D0E7E7FFFF2DE9F04FFA
:102060009A4699B0254B00248DF81C408DF81E40EF
:102070008DF840408DF84240019480460D469146CF
:1020800006930F930C4606AE04E0234600E00FAB28
:1020900034461E4601A902AA4046FFF7BEFF80F063
:1020A0000102074602A92046D2B25346C8478346DA
:1020B00038B9AC4201D100201DE0204600F01CFFE1
:1020C000F9E777B101233046214602AA00F0CAFFA2
:1020D000AC4207460CD0204600F00EFF002FD4D1B2
:1020E000E9E7AC4202D0204600F006FF012002E002
:1020F0000028CCD1DFE719B0BDE8F08F28A300009D
:1021000038B590F83E3004460D4613B1383000F033
:10211000F3FE204601212A4600F0DAFA08B9002031
:1021200038BD04F1100501222846214601F09EFA2F
:10213000024640B104F13800294600F079FD003034
:1021400018BF012038BD2846214601F08FFA00282B
:10215000E5D0EFE70A7902710A4A02604A794271D2
:102160008A7982718A688260CA68C2600A6902617B
:102170000A7D02758A698261CA69C2610A6A02625D
:10218000704700BF28A300002DE9F04F97B0054627
:10219000383104A891469A46FFF7DCFF254B4FF0F3
:1021A000000B8DF838B00D938DF83AB04C460DAF5A
:1021B00004AE2DE023782F2B01D1013428E0C4EBAD
:1021C00000085FFA88F8B8F10C0F28BF4FF00C0830
:1021D00021464246684607F0ABFB16AA02EB08030D
:1021E000384603F858BC00F087FE384631466A4648
:1021F000012300F037FF20B90E4B28712B60A87126
:1022000014E0304600F078FE334644443E461F4614
:1022100020462F2107F06AF90028CBD1C9EB04042E
:10222000CAF8004028463146FFF794FF284617B009
:10223000BDE8F08F28A30000F0B59DB004461E460F
:1022400001A86B461746FFF79FFF009BFD18FB5C3C
:102250003BB901A913A8FFF77DFF204613A91C4A2B
:1022600030E000238DF82C301A4A8DF82E309DF87E
:102270000A300A921BB92046FFF756FE24E0023BC3
:10228000012B0AA806D814492A46334600F0EAFE74
:1022900050B9F0E701A92A46334600F0E3FE0028D2
:1022A000E9D001A800F028FE16F0060F03D00AA816
:1022B000109900F0C1FD0AA913A8FFF74BFF2046B3
:1022C00013A92A46FFF704FE20461DB0F0BD00BF4B
:1022D000549E000028A3000084A3FF1F00F13803D0
:1022E000024A084619460023FFF7B8BEDD1F00006A
:1022F00000F13803024A084619460023FFF7AEBE34
:102300001120000070B504469EB00D46164628E028
:102310009DF8100000B92AE0E52822D02E2820D010
:102320009DF81B0000F00800C0B2D0B9134B8DF827
:1023300034008DF83600694604A80C9300F028FCA0
:102340000CA8E9696A46334600F08CFE78B10CA906
:1023500015A8FFF7FFFE204615A96A46FFF7B8FD4E
:1023600008E0E86904A900F01FFD0028D0DC204641
:10237000FFF7DAFD20461EB070BD00BF28A30000A5
:1023800010B50446FFF7E6FD18B1E36900229A6034
:10239000DA6010BD084B02211961084900225A7108
:1023A0009A719A721A7383F8302083F83C209963EB
:1023B00083F83E20704700BF4CA3FF1F28A30000F6
:1023C000094B1A6842F480621A602C334FF00042C5
:1023D0001A60064AFF2111601A68002AFCDA044BD1
:1023E0001868C0B2704700BF00C0024034C002404D
:1023F00038C002401A4B1B4A70B51A60C307044626
:1024000002D5FFF7DDFF013C052C01D8630800E091
:10241000032300221449154801E0086001329A4262
:10242000FBDB23EAE372A4EB42040F49104A0F4896
:10243000104D06E0166816F0F00FFBD008602E680D
:10244000023C002CF6D106E0106810F0F00FFBD033
:102450000868013B01E0064A0649002BF4D170BD33
:1024600000C0024000041F8034C00240FFFF009003
:102470002CC0024038C00240074B1A6842F4806208
:102480001A602C334FF000421A60044A10601A6838
:10249000002AFCDA704700BF00C0024034C002408E
:1024A00013B5114C052813D8DFE800F00303060923
:1024B0000C0F01A80D490DE001A80D490AE001A883
:1024C0000C4907E001A80C4904E001A80B4901E010
:1024D0000B4901A800230122FFF7DAF9019B2360D1
:1024E000FFF726FC1CBD00BFACA3FF1F00366E012A
:1024F00000127A0000093D00C0C62D0080841E0035
:10250000801A060010B5194B1B780BB3DA0707D5F4
:10251000174A1849146809682140174C2160116056
:1025200003F00202D2B23AB1144A1249146849685F
:102530002140114C6160116003F00403DBB23BB138
:102540000F4B0C4A196892680A400B498A601A605E
:102550000C4A1368834208D00B4B0C491960106079
:1025600040F0804050600A4A1A6010BD48A3FF1F27
:1025700080E100E030A3FF1F3CA3FF1F84E100E0E7
:1025800088E100E00CC0024000C0024001401F0092
:1025900000001F800C4B1B78ABB1D90703D50B4A49
:1025A00011680B4A116003F00202D2B21AB1074A55
:1025B0005168084A116003F00403DBB21BB1034BFE
:1025C0009A68054B1A60704748A3FF1F3CA3FF1F82
:1025D00000E100E004E100E008E100E008B50121CD
:1025E000007901F0CDFDFFF7D5FF08BD054B10B513
:1025F00004461868FFF786FF20790021BDE81040E7
:1026000001F0BEBDACA3FF1F10B5837904468BB1AA
:10261000008940F20123984207D8C0F500700230CB
:10262000FFF7E8FE40F2022323812046FFF7D6FFA2
:102630000023A37110BDFFFF73B50B4B1A68009206
:10264000009E0D461C46B6B2FFF7BAFEFF2808D022
:1026500023680193019B9BB29B1BAB42F4DB0020E0
:1026600000E001207CBD00BFB4A6FF1FF8B5054601
:102670000E461746FFF7C8FF2846FFF7B7FF4FF48F
:1026800096712846FFF7D8FF46F04000FFF7F4FEAA
:10269000182427FA04F0C0B2083CFFF7EDFE14F14D
:1026A000080FF6D126B1082E0CBF8720FF2000E0CE
:1026B0009520FFF7E1FE0024FFF782FE0306E87293
:1026C00004D5FF2C02D00134E4B2F5E7F8BDFFFFDA
:1026D0002DE9F04300230373837283714371544BDC
:1026E000027185B01B680446019310460F46012114
:1026F000019E01F071FD0121207901F041FD4D4B5A
:102700001A6842F480521A600620FFF7C9FE4A4B4D
:102710001868FFF7F7FE0A25FF20013DFFF7ACFE22
:1027200015F0FF05F8D1FFF735FF2046FFF75EFFF4
:10273000DFF8FC801FFA86F90BE0D8F8003002932E
:10274000029B9BB2C9EB0303B3F5FA6F01DD0123D2
:102750004EE0002120460A46FFF788FF0128054683
:10276000E072EAD1204608214FF4D572FFF77EFFD0
:1027700000F00400C0B208B125730DE00425FFF796
:102780001FFE013D15F0FF05E072F8D1AA284FF0B9
:10279000020300D02CE02373257BDFF89480022D08
:1027A0000CBF4FF080450025B6B20AE0D8F80030E3
:1027B0000393039B9BB29B1BB3F5FA6F01DD0823C8
:1027C00016E0372100222046FFF750FF2A46204618
:1027D0002921FFF74BFF0246E0720028E6D1237B58
:1027E000022B15D120463A21FFF740FF10B10623F6
:1027F000637115E0FFF7E4FD00F0C000C02801D1CF
:1028000003232373FFF7DCFDFFF7DAFDFFF7D8FDA5
:102810002046FFF7E3FE3846FFF742FE012003E0C3
:102820002046FFF7DBFE002005B0BDE8F08300BFC7
:10283000B4A6FF1F3C800440ACA3FF1F73B5114B2F
:102840001A680092009E04461D46B6B209E02B6845
:102850000193019B9BB29B1BB3F5967F01DD0F2378
:1028600007E0FFF7ADFDFF28E072F0D0FE2806D0AC
:102870000D2320466371FFF7B1FE002000E0012028
:102880007CBD00BFB4A6FF1F2DE9F843089D044698
:102890000F4690461E4603B974E09B18B3F5007FBF
:1028A00073DC83792BB10368994202D10389934287
:1028B00016D9237B2760032B18BF7F023A46204698
:1028C0001121FFF7D3FE074610B1032363715CE0CB
:1028D0002046FFF7B3FF002857D001232781A371BB
:1028E0004046FFF787FD2C492C4B1960F107324613
:1028F00004D5FFF765FD05F8010B721E052A01D806
:10290000530800E0032300212548264F01E007601B
:1029100001319942FBDBA2EB4302AA182248204F67
:10292000DFF880C0DFF884800DE0016811F0F00F5F
:10293000FBD0C7F800C0D8F80010C1F3072985F80C
:102940000090697002359542EFD302EB43031748BC
:10295000154A09E0116811F0F00FFBD00168C1F3CE
:1029600007272F70697002359D42F3D32389F6182B
:10297000A37AB6B2268113B1B6F5007F02D3204602
:10298000FFF742FE0120BDE8F8832046FFF726FE50
:102990000020BDE8F88300BF00041F8000C0024093
:1029A00034C00240FFFF00902CC0024038C00240FB
:1029B00007B54FF4007300920022FFF765FF0EBDCC
:1029C0002DE9F04104462B482B4F03682B4D43F46F
:1029D00080634FF0004603603E6029603946002363
:1029E00007468C46D1F800E0BEF1000FFADA12E09B
:1029F000D1F800E0BEF1000FFADA18E01E4A1368C1
:102A0000002BFCDA26E0112320466371FFF7E6FD78
:102A10000020BDE8F081D0F8008012F803E048F40F
:102A20008068C0F800800E60C5F800E0E0E702EBC7
:102A3000030ED7F800809EF801E0023348F4806866
:102A4000B3F5007FC7F80080CCF80060C5F800E05F
:102A5000C8D1D3E7FF20FFF70FFDFF20FFF70CFDE4
:102A6000FFF7AEFCE07200F01F000528CBD101207B
:102A7000BDE8F08100C002402CC0024034C00240DA
:102A800070B50B460446164609B9122329E0027BAD
:102A9000032A18BF4B021A461821FFF7E7FD054627
:102AA00008B104231DE02046FE213246FFF788FFCF
:102AB00088B120464FF41671FFF7BEFD08B9152303
:102AC0000FE020460D212A46FFF7D0FD40B9FFF761
:102AD00077FC28B907E02046FFF780FD002070BD95
:102AE00014236371F7E72046FFF778FD012070BDDE
:102AF000014A024B1A60704701100138ACA3FF1F56
:102B000010B504460121006A04F1080200F032FD0C
:102B100040B1E3692BB9A368E361637963F07F0394
:102B20006371012010BD70B50446FFF7E9FF08B9D5
:102B3000002070BD236AA268197C1D79023A02FA4E
:102B400001F65A69B218561E06E0701900F056FCDC
:102B50000028EDD0013DEDB2002DF6D1236A1B7C9B
:102B60004FF4007202FA03F2A3699B18A3610120DB
:102B700070BDFFFF10B50446006900F01BFC18B1E2
:102B8000207D024B03EB401010BD00BFBCA3FF1F14
:102B9000002230B513462E24855C202D09D0D5B2F5
:102BA000082D02D1CC540133DBB2855CCD54013306
:102BB000DBB201320B2AEFD10022CA5430BDFFFF35
:102BC00070B5002305462022CA5401330B2BFBD1DC
:102BD000002207241FE02E2B01D0144E06E00A2C01
:102BE00022D008220A2416E098421DD016F8010FC0
:102BF0000028F9D1A24218D8202B16D97E2B14D840
:102C0000A3F16106192E01EB020001D8203BDBB2D3
:102C100001320370D2B215F8013B002BDBD10878EA
:102C2000203818BF012070BD002070BD0FA3000028
:102C300038B5827904460D460AB1002038BD91F8B6
:102C40002030102B06D1022383714B8CC2615B01B3
:102C500083610CE0202BF0D103238371496A04F1D6
:102C60001802C161284600F019FC0028E5D00023B5
:102C7000012025626071A360E3602361237538BD84
:102C80002DE9F04F837985B00446904613B94FF68D
:102C9000FF7865E04379DB07F9D564E01FFA83F834
:102CA00047460E46DFF8F890DFF8F8A056E0E268F5
:102CB000A179206AD3054FEAD35B02291FFA8BF36F
:102CC0004FEA522E02D1416A71441CE00579013D60
:102CD00005EA0E05EDB26BB965B912B9E269A260F9
:102CE00008E0A168039304F1080200F0A3FB039B32
:102CF0000028CCD0226AA168107C5269023901FAFE
:102D000000F189184919CBF500729742627902F0F7
:102D10004002C8BFC3F50075D2B2CCBFADB23D46CC
:102D200012B9B5F5007F2ED1DAF80020914220D1FA
:102D300029E076190DE00BEB090358191A463146C4
:102D400003E012F801CB01F801CB8242F9D1D31A8A
:102D5000F618E3687F1B5B19E360BFB2002FA6D1B2
:102D60000FFA88F016E08269C368D31A984595D89F
:102D700096E70A4A009610681A462B46FFF784FD2C
:102D80000028D6D183E70846002100F013FB002875
:102D9000D1D17CE705B0BDE8F08F00BFB8A3FF1F1D
:102DA000BCA3FF1FA08FFF1F38B58379012B0546F9
:102DB0000C4601D8FF201BE0C368DA06FAD10AE00E
:102DC0002278A2B1E52A06D02E2A04D0E27A02F0B7
:102DD0000802D2B262B1202228462146FFF750FFF6
:102DE00042B2202AECD0002AE4DB002000E01046AA
:102DF00040B238BD37B58379012B044601D8002095
:102E000016E0C36801220DF10701C3F34315FFF774
:102E100037FF01280CBF9DF807304FF6FF731BB238
:102E20000133ECD0E26803481F32E26000EB45104A
:102E30003EBD00BFBCA3FF1FF8B5044680790D4618
:102E400000282CD0A369994224D825E01DB9A5609B
:102E5000E5600120F8BD236AE2681E7C691E093620
:102E6000531E23FA06F321FA06F69E4200D312B946
:102E7000E369A36009E0F61A07E0206AA1683A4610
:102E800000F0D8FA013E10B9F8BD04F10807002E91
:102E9000F3D1DDE70020F8BD0228D7D1D8E7F8BD8F
:102EA00038B58379054613B390F90530002B1ADA4B
:102EB0000121FFF75FFE0446C8B1AB79012B9CBF2F
:102EC000AB69C361EB6943831B0C8382094B1B68AD
:102ED0002BB1183004F116019847238B63826B796C
:102EE00003F07F036B71BDE8384000F03DBA00206D
:102EF00038BD00BFB0A3FF1F10B50446FFF7D0FFD9
:102F000010B10023A371012010BDFFFFF7B5827936
:102F1000012A04460D4645D1437903F00203DBB292
:102F2000002B3FD040E0002B3AD0E668FFF784FF4B
:102F300000B937E0206A35B9E16900F073FB002879
:102F400030D0E5611BE0A16801AA00F073FA48B334
:102F5000206A184B90F8207001994FF6F872102FE4
:102F600008BF134699420AD200F05CFBD0B1206A38
:102F7000A1686FF0704200F0B9FA00B912E063790D
:102F8000A56163F07F0363712046FFF789FF48B1B5
:102F90002046B54234BF29463146FFF74DFF07E0D2
:102FA000104605E0002003E083699942BBD9F9E7A8
:102FB000FEBD00BFF8FFFF0F10B500210446FFF76C
:102FC000A5FF60B120460121FFF7D4FD38B1E5230C
:102FD00003700023A371BDE8104000F0C5B90020C4
:102FE00010BDFFFF38B51D4B03EB41131546DA7AD0
:102FF00012F0110F044604D015F0420F01D000204A
:1030000038BD174A2175126822615A8B998A42EAA3
:103010000141E161DA7A12F0180203D1DB69A361A0
:10302000012309E0102AEAD1206A04F1180200F015
:1030300035FA0028E3D00423A37105F00F0305F04F
:1030400040050021EDB26371A160E16025B1204629
:10305000BDE83840FFF75ABF012038BDBCA3FF1FB1
:10306000A08FFF1F2DE9FF47867905460C461F46B6
:10307000002E75D10DF1040810464146FFF7A0FD62
:1030800000B96DE0236AA6602B62E660DFF8E0908D
:10309000C24621E02046C3F34318FFF7ABFE0146CA
:1030A00000285DD002780AB1E52A09D126B9D9F8FD
:1030B000002085F814802A610B78012683B10BE08B
:1030C00050460B2205F052FE30B907F03003302B8A
:1030D00046D0284641463FE0E368A2699342D9D3EF
:1030E00007F01203122B3BD136B128460121FFF71E
:1030F00041FD044648B933E0A379022B30D0204685
:10310000FFF711FD60B3184C2E75002120222046D8
:1031100001AE05F07DFF03CE20606160B378328898
:10312000A372124B22811B682BB104F1100004F131
:103130000E01984706E021222274A3732822082357
:103140006274E373238A63822383E389E38200F05A
:103150000BF928B1297D28463A46FFF743FF00E0E6
:10316000002004B0BDE8F087BCA3FF1FB0A3FF1F81
:10317000A08FFF1F10B50A468AB0094900230446F4
:103180008DF8083001918DF80A3001A821460223FC
:10319000FFF768FF10B101A8FFF70EFF0AB010BDDE
:1031A00028A300002DE9F74F92468279012A0746AD
:1031B0000C4640F0B680427902F00201C9B2002903
:1031C00000F0AF80B1E0B969FD688D4201D155468C
:1031D00088E0FFF731FE002800F0A380F7E7386AA7
:1031E00090F804B00BF1FF3B0BEA522B4FEAC259A7
:1031F0004FEAD9591BF0FF0B1FFA89F81FD1B8F11C
:10320000000F1CD1B96811B9FA69BAB911E001AA65
:1032100000F010F9002800F08F80396A474891F8D3
:103220002010019A4FF6F873102908BF1846824201
:1032300004D33846FFF764FC08B972E0BA603A6A12
:10324000B968107C5269C8F500760239B6B2B54249
:1032500038BF2E4601FA00F18918B6F5007F8B447D
:1032600011D1374A1168594504BF4FF0FF31116041
:10327000344A594610682246FFF702FC002850D015
:1032800004F5007429E0B8F1000F10D1F968BA69AB
:1032900091420CD300F068F8002842D0284AC2F8C6
:1032A00000B0294A117841F00101117005E058463B
:1032B000012100F07FF8002833D0244A914409EB23
:1032C0000600611E4A4603E011F801CF02F801CB67
:1032D0008242F9D1C9EB02094C44FA68AD1B961938
:1032E000ADB2FE60FA68002D7FF479AFB9698A4209
:1032F00001D9BA6105E0164A126832B1BAF1000F7D
:1033000003D07A7962F07F027A717A7902F008024A
:10331000D2B20AB950460FE03846FFF7C1FD002887
:10332000F8D101223A71002006E002F00402D2B284
:10333000002A7FF448AF4AE7BDE8FE8FF8FFFF0F91
:10334000A08FFF1FB8A3FF1FBCA5FF1FBCA3FF1FBB
:10335000B0A3FF1F07B502AB012203F8011D1946F8
:10336000FFF720FF0EBDFFFF38B50D4B1B78A3B153
:103370000C4D0D4B286819680C4AFFF781FB68B1AA
:103380000B4C216831B12868084AFFF779FB28B156
:1033900000232360024B00221A70012038BD00BFB9
:1033A000BCA5FF1FB8A3FF1FA08FFF1FBCA3FF1F5B
:1033B000B4A3FF1F70B50D4D2B68834204460E4623
:1033C0000DD0FFF7D1FF08B9002070BD084B094AA6
:1033D00018682146FFF7ECFA0028F5D02C60064B60
:1033E0001A7816431E70012070BD00BFA08FFF1F0A
:1033F000B8A3FF1FBCA3FF1FBCA5FF1F10B5044649
:10340000FFF7B2FF78B10023074A194699540133F8
:10341000B3F5007FFAD1054B1C60054B1A7842F0DA
:1034200001021A70012010BDBCA3FF1FA08FFF1F57
:10343000BCA5FF1FC3680133994270B505460C4611
:10344000164601D9002070BD95F82030C069102BB8
:1034500001D10B0A00E0CB0918180E4B1B689842EB
:1034600005D195F82030102B0B4B0AD105E0002137
:10347000FFF7A0FF0028F4D1E4E7E4B233F81430FA
:1034800005E004F07F0453F8243023F070433360E8
:10349000012070BDA08FFF1FBCA3FF1F2DE9F743C4
:1034A00002AEDFF8448046F8041D054617460024A6
:1034B0004FF6F879284601993246FFF7BBFF80B1F5
:1034C0002B7C4FF4007202FA03F395F82020E418E5
:1034D000019B102A14BF42464A469342EAD33C60FD
:1034E0000120BDE8FE8300BFF8FFFF0F0129F8B5FA
:1034F00004460D46174633D9C368013399422FD885
:1035000090F82030C669102B01D10B0A00E0CB09DE
:103510009E19144B1B689E4205D194F82030102B45
:10352000114B0BD106E030460021FFF743FF002886
:10353000F3D1F8BDEDB223F8157003E005F07F0577
:1035400043F82570094B1A7842F001021A70237E65
:10355000012B03D9A368F618054B1E600120F8BDA6
:103560000020F8BDA08FFF1FBCA3FF1FBCA5FF1F3D
:10357000B4A3FF1F2DE9F74F156806468A46174684
:103580001DB101354FF0000905E04B1ED3F10009D4
:10359000056859EB0309F3682C4603F1010B4FF062
:1035A0000008F36898451CD25C4501D902242546E1
:1035B0003046214601AAFFF73DFF90B1019A631CF6
:1035C0000AB11D4602E05B1B534503D008F1010818
:1035D0000134E6E7304621466FF07042FFF786FF80
:1035E00058B900201CE004F1FF383046414622461D
:1035F000FFF77CFF0028F4D04446AC42F3D839688A
:1036000021B93D60B9F1000F07D108E030462A46E4
:10361000FFF76CFF0028F4D1E3E7013535600120A6
:10362000BDE8FE8FF7B502230F4F036005460C4639
:103630004FF6F8762846214601AAFFF7FBFE80B137
:10364000284621460022FFF751FF50B195F820305F
:10365000019C102B14BF3B4633469C42EAD3012009
:1036600000E00020FEBD00BFF8FFFF0FF8B53B4BA8
:10367000044619601546CAB1042A01D90020F8BDD4
:1036800000200146FFF796FE0028F7D0344B03EBED
:10369000051505F5D475AA795206EFD1D5F8122093
:1036A000632AEBD9D5F80E50002DE7D0284600212B
:1036B000FFF780FE0028E1D0294BB3F80B20B2F5CC
:1036C000007FDBD11A7C002AD8D0D9890029D5D037
:1036D0005B7B002BD2D02276002223712274012042
:1036E00003E0511C072A2174C8D8227C00FA02F199
:1036F0008B42F6D11A4BD98A01B9596ADE89A16089
:10370000AE19E661B3F811001F7C6084400107FB2D
:10371000016100F2FF10616201EB50216161B3F8B9
:1037200013300BB90E4B1B6A691ACB1823FA02F23D
:1037300040F6F4739A42E26001D80C2309E04FF698
:10374000F4739A4201D8102303E0054BDB6A6362ED
:10375000202384F820300120F8BD00BFB8A3FF1F4C
:10376000BCA3FF1F094B1B7813B9094B1B782BB166
:10377000084A1378202B03D90123037100207047D6
:103780000548C154013313700120704722A6FF1F62
:10379000E5A5FF1F23A6FF1FC4A5FF1F7047FFFF5E
:1037A000024B1878024B1B78C01A704721A6FF1FE6
:1037B00020A6FF1F064A074913780978994204D9C1
:1037C0000549C85C0133137070474FF0FF307047F4
:1037D00020A6FF1F21A6FF1FE6A5FF1F054B064AD7
:1037E0001B7812789A4202D9044AD05C70474FF095
:1037F000FF30704720A6FF1F21A6FF1FE6A5FF1F71
:1038000038B50E4B1B78144613B90D4B1B788BB192
:103810000C4B1D78C5F121039C4202D90122027193
:103820001C4609482246401905F0D2FA054B2D19CD
:103830001D7000E01C46204638BD00BF22A6FF1FB9
:10384000E5A5FF1F23A6FF1FC4A5FF1F10B5104B42
:103850001B7813F020040BD1122000F045FB0D4B18
:103860001B68A3B10C4A14700C4A1078984710BD1D
:103870000B4A13780133DBB2012B137002D8094BCA
:103880001B7823B91220BDE8104000F02DBB10BDFD
:1038900003600640C0A5FF1F20A6FF1F21A6FF1F33
:1038A0000CA6FF1FE5A5FF1F002202710273034A49
:1038B0004FF47A7181600260704700BF38A3000046
:1038C00010B5374A137803F01001C9B221B903F0DB
:1038D0004002D2B242B92EE01021117003F0400232
:1038E000D2B2002AF3D110BD13F004032D4A18D030
:1038F000002313702C4A13702C4B1B68144603B121
:10390000984722782A4B1AB927491A700120087063
:10391000284AD02111701A78274B1A700122274BA0
:1039200021E001211170264A1370224BC0221A7027
:1039300002331B7830E01F4A1F4C117811F0100140
:1039400017D013F0010310D11C4917480A780078EA
:10395000904205D9164B9B5C013223700A7000E03F
:103960002370144BD0221A7016E0C02313702378F2
:1039700012E0144B122019700322134900F08AFA46
:103980000F4A207813781F2B06D80649097819B1F9
:103990000E49C85401331370014B02221A7010BD36
:1039A00003600640BDA5FF1F23A6FF1F08A6FF1F3B
:1039B000C4A5FF1F026006400460064024A6FF1F46
:1039C00021A6FF1F0CA6FF1F4D380000E6A5FF1F14
:1039D0000148FFF769BF00BF10A6FF1FF0B53048D0
:1039E000304903681B06FCD40B6813F08002F8D141
:1039F00072B62D4B1978002950D02C4908684F68B1
:103A00008E68CD680C69381814318019096840191E
:103A100000194018C0F34E00254940F400400860EA
:103A2000C86A0F6B4E6B8D6BCC6B381840318019A8
:103A30000968401900194018C0F34E001D4940F4B0
:103A40000040086001F10811143151F8140C51F8CC
:103A5000107C51F80C6C51F8085C51F8044C096862
:103A600038188019401900194018C0F34E00124947
:103A700040F400400860C86A0F6B4E6B8D6BCC6BD6
:103A80003818403180190968401900194018C0F3EE
:103A90004E000A4940F4004008601A7062B6F0BD5A
:103AA00024B0034024B00B4026A6FF1F38B00340CB
:103AB0002CB0034030B003402CB00B4030B00B4072
:103AC000224B60221A70E1225A70214B214A197848
:103AD000214B082901D1012102E00A2907D139210E
:103AE000116013221A601D4B19605A600BE00C29FB
:103AF0001A4901D1352000E03D20106012221A60E1
:103B0000174B08601A60174B17491B78174A03B107
:103B100001230B601360164B164A1978164B0129C6
:103B200001D880210CE0042901D8842108E008296B
:103B300001D8852104E0102901D8862100E08721E1
:103B4000116019600D4B01221A7070470040074048
:103B5000A48FFF1F08B003400CB0034008B00B4017
:103B60000CB00B4029A6FF1F20B0034020B00B4033
:103B7000A58FFF1F24B0034024B00B4026A6FF1FD3
:103B80000D282DE9F0410FD9172801D80E380AE089
:103B9000A0F11A03052B01D8093804E0A0F1220393
:103BA000062B4DD81838C0B2274B1C5C274B1B780E
:103BB0000BB1FFF713FF72B6200614D4244D254E27
:103BC00001272C60377062B672B62B68190603D5D0
:103BD000214B18681F4B23E03378002BF1D062B6DD
:103BE00001F084FCF0E704F040071C4D1C4EFFB2CE
:103BF00004F03F044FF001081A4B1A6817B122F085
:103C0000100201E042F010021A602C6086F8008079
:103C100062B672B62B681A060BD5134B1868104B98
:103C200000221A7062B6114B1B7840FA03F0BDE80F
:103C3000F0813378002BDFD062B601F057FCE8E763
:103C40000020BDE8F08100BF50A3000026A6FF1FA2
:103C500000B0034028A6FF1F10B0034000B00B4087
:103C600027A6FF1F0CB00B4010B00B4025A6FF1F6E
:103C7000024A1378DB07FCD5704700BF0100024001
:103C800030B5194B85B06C4603F1100518685968BA
:103C9000224603C20833AB421446F7D1134B1B78BC
:103CA00003F00203DBB2BBB1114B80221A70332246
:103CB0001A710322DA7072B60E4C6B4643F00103A0
:103CC0002046984762B6237813F0700304D023701F
:103CD00008E0013B03D105E0044944F621630A787A
:103CE000D207F6D505B030BD68A300000100024040
:103CF0000700024000000240B0F5006F10B5044616
:103D000009D2064B1B78D90701D4FFF7B9FF04F19C
:103D1000A054207810BD002010BD00BF010002405B
:103D2000B0F5006F38B504460D460FD2084B1B782E
:103D3000D90701D4FFF7A4FF04F1A0542378AB42C4
:103D400004D02570BDE83840FFF792BF38BD00BFF2
:103D500001000240024B1A6801321A60704700BF2E
:103D6000B4A6FF1F38B50B4C25462368580301D570
:103D700000F090FB2B68590501D501F0A7FD2B68D9
:103D80001A0501D501F0E0FF2368DB04EDD502F050
:103D9000B3F9EAE73480044008B5FFF7E3FFFFFF1B
:103DA000014B10221A807047002005407047FFFF2A
:103DB000024A13681818106018467047A88FFF1F32
:103DC000FEE7FFFFEFF313839BB9EFF3108098B981
:103DD000EFF3058323B10F2B04D9084A985C01E067
:103DE0004FF48070EFF311833BB1984228BF18461F
:103DF00070474FF0FF30704718467047F0E300E01F
:103E0000002300E00133C25C002AFBD11846704752
:103E100010B50023B0FBF2F402FB1400092801D80E
:103E2000303000E03730C85420460CB10133F1E7A0
:103E3000CA185470224605E0885CCC5C8C54C85487
:103E40000132013B9A42F7DB084610BD031E10B554
:103E50000C4603DBBDE81040FFF7DABF2D2001F868
:103E6000010B5842FFF7D4FF204610BD084B4FF41A
:103E700000021A604FF080721A604FF000721A60F0
:103E80004FF080621A604FF000621A60704700BF06
:103E900008E100E0212830B521D8042A1FD8DFE846
:103EA00002F00709050B03000B2306E00A2304E0D8
:103EB000082302E00C2300E00923094A02EBC002B8
:103EC000526872B61468074D24F47024146044F0EC
:103ED000807444EA034345F82010136062B630BD95
:103EE00078A300002CA6FF1F094B03EBC0035B68FF
:103EF00072B61A6822F0877222F4803242F0807221
:103F00001A60044B002243F8202062B6704700BFBD
:103F100078A300002CA6FF1F114B10B51C68E0040D
:103F20001C6004D50F4BDA680AB1DB689847A1041E
:103F300004D50C4B1A690AB11B699847A20604D52F
:103F4000084B1A6E0AB11B6E9847E30606D5054B5F
:103F5000D3F8842012B1D3F88430984710BD00BF45
:103F6000A09004402CA6FF1F1F4B10B51C68E00357
:103F70001C6004D51D4B1A680AB11B689847A10341
:103F800004D51A4B5A680AB15B689847E20704D512
:103F9000164B1A6C0AB11B6C9847A30704D5134B38
:103FA0005A6C0AB15B6C9847200704D50F4B9A6C8A
:103FB0000AB19B6C9847610704D50C4BDA6C0AB1C7
:103FC000DB6C9847220304D5084B5A6E0AB15B6E2E
:103FD0009847630306D5054BD3F8802012B1D3F878
:103FE0008030984710BD00BFA0A004402CA6FF1F42
:103FF0002C4B10B51C6820071C6004D52A4B5A6A4C
:104000000AB15B6A9847E10604D5274B9A6A0AB160
:104010009B6A9847620604D5234BDA6A0AB1DB6AC9
:104020009847230604D5204B1A6B0AB11B6B98479F
:10403000A00604D51C4B5A6B0AB15B6B9847E1078D
:1040400004D5194BDA6B0AB1DB6B9847A20704D58C
:10405000154B9A6D0AB19B6D9847630704D5124BB7
:10406000DA6D0AB1DB6D9847A00504D50E4BDA6E08
:104070000AB1DB6E9847E10504D50B4B1A6F0AB104
:104080001B6F9847620504D5074B5A6F0AB15B6FE7
:104090009847230504D5044B9A6F0AB19B6F984744
:1040A00010BD00BFA0B004402CA6FF1F1E4B10B5D2
:1040B0001C68E0071C6004D51C4B9A680AB19B6819
:1040C0009847210604D5194B5A690AB15B6998478C
:1040D000E20604D5154B9A690AB19B6998476307B4
:1040E00004D5124BDA690AB1DB699847200704D579
:1040F0000E4B1A6A0AB11B6A9847A10704D50B4BED
:104100009A6B0AB19B6B9847A20604D5074B1A6DB0
:104110000AB11B6D9847630604D5044B5A6D0AB16A
:104120005B6D984710BD00BFA0C004402CA6FF1FC8
:10413000094B10B51C68A2071C6004D5074B9A6E8A
:104140000AB19B6E9847E30704D5044BDA6F0AB1B6
:10415000DB6F984710BD00BFA0D004402CA6FF1F06
:10416000044B054900221A600A60044A10601022BC
:104170001A60704714D0034004D0034000D00340BD
:10418000212810B518D80D4A52F8303093F88042E3
:104190003CB1012211B183F8802010BD83F80021C9
:1041A00010BD02EBC00043681A6811B142F003026F
:1041B00001E022F002021A6010BD00BF78A30000E7
:1041C000212805D8034B53F8303093F8000270478C
:1041D0000020704778A30000212816D80B4A02EB74
:1041E000C00301295B6852F8302004D182F88012A4
:1041F0004FF4A27208E0002082F8800211B94FF457
:10420000807201E040F203121A60704778A3000048
:1042100072B60B4B0B491A680B4B1B68096862B6E8
:10422000490102D5322A88BF0133C2F5BB32FF32C1
:104230006021B2FBF1F24FF47A7000FB032070476B
:1042400018E000E004ED00E0B4A6FF1F70B50446DE
:10425000FFF7DEFF05466CB140F2E736FFF7D8FF07
:10426000401BB04203D9013C04D005F57A7501F03A
:104270003DF9F3E770BDFFFF10B5FFF7F7FD164BF3
:10428000164A174C00204BF6FF711860596028231E
:10429000136093601361936113629362136393637A
:1042A000092222600F4C20606160A360236144F802
:1042B000042C0D4C20600D4801600D490B608B6093
:1042C0000C4B1A60FFF7FCFB0420FFF7BFFFBDE8B3
:1042D000104000F0FBBB00BF048003400C80034093
:1042E000008003400490034004800B4008800B4092
:1042F0000C800B4000800B40F0B50C4B0C4C1A7836
:1043000042F0020504EBC50682F001027060094824
:104310001A700678002E0CBF8827C82747EA01418B
:1043200086F0010644F835100670F0BD20A7FF1F87
:104330000080FF1F98A7FF1F431E032B10B510D846
:1043400072B6094A52F8230048B1416842F8231076
:10435000064A018832F81340611A22F8131062B637
:1043600010BD002010BD00BF10A7FF1FC8A9FF1F70
:10437000013803280BD872B6064B53F820300020C2
:1043800001E05B680130002BFBD162B67047002072
:10439000704700BF64A7FF1F70B572B6184E194C66
:1043A00001239A1912F8012C02F00802D2B2E2B1EC
:1043B0009900144A54F831502DB902EB43130830D8
:1043C0005860114B09E041F0010154F8315065B9D2
:1043D00002EBC103083058600C4B42F831300C4BF3
:1043E0001A78013A1A7062B670BD0133052BD8D124
:1043F00062B6074B00221A70BDE8704000F0D2BBD5
:10440000B0A400000080FF1F88004000C8004000EA
:104410008EA7FF1F431E032B30B532D84001194A27
:1044200040F01000101872B6174CE25C032A09D84D
:10443000DFE802F0160218050830022213E0083007
:10444000042210E01148124A50F8234014B940F8F1
:10445000231002E052F82300416042F823100FE0DD
:10446000032200E00522E25410F0080F01F10803D6
:104470000A8843600CBF8823C82343EA02430360D1
:1044800062B630BD0080FF1FCCA6FF1F64A7FF1FD0
:1044900074A7FF1F2DE9F74FA54EA64C357805F000
:1044A0000403DBB2ABB1A44B1B7883B1A34A1378EE
:1044B00023B1013BDBB2137003B900BEA04A1378ED
:1044C0002BB1013BDBB213700BB900F07FFC04236E
:1044D000337005F00802D2B2002A00F08082994BB6
:1044E0001B781D094FEA930940F0FE8104EBC903D4
:1044F000586854F83930C3F38303013B0C2B00F2A6
:10450000F081DFE813F0A901A901EE01EE01EE014F
:10451000EE01EE01EE01C501EE01EE01EE010D002E
:104520004368894902684B60884B894844F83930B0
:10453000884D0A60002303600120287092B240F287
:104540008165AA422361A36117D8B2F5D06F80F0CC
:104550002C81B2F5817F00F0DC8006D8802A00F043
:10456000C280822A40F03D81C1E040F202339A428B
:1045700000F00C81B2F5A06F16E042F22105AA42CC
:1045800000F0678108D8B2F5086F00F0A680B2F598
:10459000106F40F026810AE042F22120824200F0B2
:1045A0001C8142F221339A4240F01B811DE18A783E
:1045B000614B604D1A702B6A180603D5686A08387B
:1045C00000F0F0FA644A08359542F4D1DFF8B09172
:1045D000DFF8B0B10025A846CA4655F8090005E045
:1045E0004368009300F0DEFA009B18460028F7D1DC
:1045F0005A4B4AF8050045F80B00E85807E04268B6
:104600000093019200F0CEFA019A009B1046002818
:10461000F5D15851524BE850524B23F81800524BE9
:1046200018F80320023A032A08D8DFE802F002044F
:104630000204002200E0012203F8082008F101082A
:104640000435B8F1040FC8D1484BDFF83C91002283
:104650001A7001259846464B05EB0902EB1812F833
:10466000012C9B001A7002F00802D2B23AB300F09B
:104670007BFAAB0038B104EB4512083050603D4A7C
:1046800044F8332006E044F8330098F80030013352
:1046900088F8003000F068FAAB0043F0010338B14D
:1046A00004EBC30208305060284A44F8332006E087
:1046B00044F8330098F80030013388F80030AA003D
:1046C00042F00201013542F003020023052D44F8B7
:1046D000313044F83230BED188E0174B264D1B787C
:1046E0002B70034685E0244D2B706B7080E08A8828
:1046F000042A00D975E0204D2B706B701F4B92007F
:10470000D3181B7803F00203DBB2002B70D02870A3
:104710006EE08A8802F07F03042B62DC4B8803B1D1
:104720005FE09100154A8A18117821F0020156E0E5
:10473000802007400080FF1F97A7FF1F21A7FF1FB2
:1047400099A7FF1F9020074084A7FF1FC8004000C3
:10475000B8A6FF1F98A7FF1F8080FF1F64A7FF1F39
:1047600074A7FF1FC8A9FF1FCCA6FF1F8EA7FF1F9E
:1047700030C80110880040008FA7FF1FC0200740ED
:1047800010A7FF1FBCA6FF1FB0A400008A8802F07C
:104790007F03042B25DC4B8803B122E09100A14A62
:1047A0008A18117841F0020119E04A889E4B8988E5
:1047B00053F8085CA3F10C009DB133F80CCC944580
:1047C00009D133F80ACC8C4505D1120A032A0CBF53
:1047D0002B7803890DE00C33EAE78978934A11704E
:1047E00004E0904B0F221A7033E000231D4600E0D6
:1047F00002238F4AB2F806904B4538BF9946B9F16B
:10480000400F34BFC8464FF0400828464146FFF7E6
:1048100073FDB9EB0809454403D1B8F1400F07D047
:1048200017E0B9F1400F34BFC8464FF0400800E030
:10483000C84628464146FFF75FFDB9EB08094544E5
:1048400002D1B8F1400F04D17A4B7B4A1D60A2F827
:1048500000900122794B43E0754B1A8842F2210304
:104860009A4211D1764A0023C15C99540133072B37
:10487000FAD1734B1B68862B02D1724B0F221A7030
:1048800000200146FFF738FD6F4B44F8393028E02F
:10489000684BD3F80080B8F1000F18D0DFF898917A
:1048A000B9F800A0BAF1400F34BF55464025404644
:1048B0002946FFF721FDC5EB0A039BB2A9F800309A
:1048C0000BB9402D01D108EB05035A4A1360584B30
:1048D0001A88B2F5A06F04D100225A709A785B4B07
:1048E0001A700122554B6DE004EBC90803F0080370
:1048F000D8F80420013DD9B2A2F10800EDB2002998
:1049000037D000F04FF95248524B50F82510F1B112
:104910004A6840F8252001F10802C8F804205A5DD1
:10492000032A0BD8DFE802F002040608032204E0A1
:10493000022202E0052200E004225A5518F0080F76
:104940000A880CBF8823C82343EA024342E05A5D29
:10495000032A07D8DFE802F040400204002206E004
:10496000012204E018F0080F0CBF022203225A555E
:1049700032E054F839301B0C22F8083C23B322F8FB
:10498000061C42F8041C344A344952F8257017B901
:1049900042F8250002E051F825205060304A41F8E5
:1049A000250032F815105B1822F8153000F0DCF8FD
:1049B00018B10830C8F8040006E02A4B44F8390062
:1049C0001A7801321A7007E01F4B274A18F0080FB7
:1049D00008BF134644F83930082333705EE5E90711
:1049E00052D516492048214C02230B70204B1A70D7
:1049F000204B1860986020481A61D8609A615C600A
:104A0000084B0D2018701D48FF23037000F8083C68
:104A100002741B4A13701B4B9F221A7001230B70E8
:104A20004BE000BFC0200740C0A40000A8A7FF1FA4
:104A300084A7FF1FB8A6FF1F8CA7FF1F9420074065
:104A4000D0A9FF1F21A7FF1FC800400098200740E2
:104A500064A7FF1FCCA6FF1F10A7FF1FBCA6FF1F48
:104A6000C8A9FF1F8EA7FF1F88004000D0A6FF1F08
:104A700020A7FF1F0080FF1F24A7FF1F88200740DB
:104A80008C200740842007402B0605D50C4B0D22B7
:104A90001A70802203F8402C05F00203DBB22BB120
:104AA000084B1A781A70022203F8082C05F010053A
:104AB000EDB215B1044B10221A70BDE8FE8F00BF95
:104AC000C0200740882007408020074008B501F03B
:104AD00069FB00231E491A465A50C8180833882B10
:104AE0004260F9D11B4B1A6842F480221A601A4BBB
:104AF00080221A701978184A0906FBD4144B1749FA
:104B0000C3F307200870C3F307401B0E08750B762C
:104B1000FF2301F81C3C01F8143C01F88C3C13788D
:104B200043F0400313700021012302F8783C02F89F
:104B30000C1C02F8883C0A4B70226FF4507C1A70EF
:104B400063444FF400721A60064B10221A7008BDBD
:104B50000080FF1F348004400C2107409C20074048
:104B600049E400E00821074072B60C4A1168B1FA26
:104B700081F30B2B02D962B6002070474FF0004042
:104B800020FA03F021EA0001116062B604494822CC
:104B90005343C8180022CA5042607047AC8FFF1FB1
:104BA000008CFF1F0C4B4822C31AB3FBF2F30B2BF4
:104BB00011D80A4A127822B1094A12780AB1FFF7CD
:104BC000EBBB72B6074A4FF0004121FA03F31168BC
:104BD0001943116062B67047008CFF1F8EA7FF1F3C
:104BE00097A7FF1FAC8FFF1F38B5114C23684BB13F
:104BF0000F4D28684288811801320C7A01888A4258
:104C000012D30CE00B4B1B7813B94FF0FF340CE0C0
:104C10000320FFF791FB20600028E9D1F5E7FFF7BB
:104C2000C1FF00232B6000E04280204638BD00BF5A
:104C3000A4A7FF1F97A7FF1F10B50C4C23681BB13B
:104C40000A4B1B686BB902E0094B1B7813B94FF094
:104C5000FF3010BD0320FFF76FFB20600028EFD16D
:104C6000F5E75A889B18187A10BD00BFA4A7FF1F4C
:104C700097A7FF1F044B9888044B1B681BB11A8829
:104C80005B88D31AC0187047C8A9FF1FA4A7FF1FCD
:104C90002DE9F8432D4B2E4DDFF8C08001220C4644
:104CA0001A7006464BE02B682BBBDFF8A0904AF247
:104CB000F92798F8003013B9244A137014E004203F
:104CC000FFF756FB072808D8012389F80030FFF7C3
:104CD0004BFF286078B989F80000013F1D4B01D0D7
:104CE0001A782AB101221A704FF0FF30BDE8F8831C
:104CF00000F0FCFBDDE72968164A488800231370A2
:104D0000C0F14002944238BF224600F108078018E3
:104D1000CF194880A41A02E0F05CF85401339342A2
:104D2000FAD1F6184B883F2B06D940230B8004207C
:104D3000FFF770FB00232B60074B05221A70002C35
:104D4000B1D1024B20461C70BDE8F8839AA7FF1F23
:104D50009CA7FF1FA0A7FF1F99A7FF1F97A7FF1FD3
:104D600007B502AB012103F8010D1846FFF790FFCC
:104D70000EBDFFFFF8B5114B1B78EBB1104E114B78
:104D80003468114D01271F704CB1638800272F70C4
:104D9000042023802146FFF73DFB376009E0FFF741
:104DA000E3FE014620B104202C70FFF733FB00E046
:104DB0002F70044B00221A70F8BD00BF97A7FF1F89
:104DC0009CA7FF1F9AA7FF1F99A7FF1F38B50D4B80
:104DD0001D78ADB90C4C216831B14B8804200B8093
:104DE000FFF718FB256038BDFFF7BEFE014620B176
:104DF0000420BDE83840FFF70DBB044B01221A70B8
:104E000038BD00BF9AA7FF1F9CA7FF1F99A7FF1FD0
:104E1000F0B5C02928BFC02172B6124B1860124BE2
:104E200000221A605A609A60DA601A615A6101269B
:104E30000AE0540902F01F0753F8245006FA07F756
:104E40003D4343F8245001328A42F2D100234FF40B
:104E5000817203E002FB0304637001338B42F9D1DA
:104E600062B6F0BDB4A7FF1FBCA7FF1F10B572B696
:104E70001E4B1868A0B9586850B9986850B9D868DE
:104E800050B9186950B95869143348B962B610BDA1
:104E9000043305E0083303E00C3301E01033FFE78F
:104EA000B0FA80F14FF0004222FA01F220EA02004B
:104EB00018600F4802780132D2B2027062B60B4815
:104EC0001B1A9B105B01591A4FF481734B4309491C
:104ED00003F5F9531E3309680124CC54C818064B56
:104EE0001978914238BF1A7010BD00BFBCA7FF1FD0
:104EF000B9A7FF1FB4A7FF1FB0A7FF1F417872B665
:104F00000378012B02D9013B037011E04A11094BD0
:104F1000C9434FF0004001F01F0120FA01F153F89E
:104F20002200084343F82200034B1A78013A1A7012
:104F300062B67047BCA7FF1FB9A7FF1F30B5C36893
:104F40000EE0187A90420AD158685C7A006950F8ED
:104F5000245025B940F82410087801300870DB6827
:104F6000002BEED130BD437A99424FF0000305D2B9
:104F7000026952F8210042F8213070471846704704
:104F800038B5437A994201D3002418E0036953F8F5
:104F90002140002243F82120002CF5D02378012B5A
:104FA0000DD9FFF763FF054628B10230A11C4FF46D
:104FB000807203F00DFF2378013B23702C462046BE
:104FC00038BD10B54168427A4B7A9A420ED872B613
:104FD0000268D36813B9D06004E02346DC68002C73
:104FE000FBD1D860012313720B7262B610BDFFFFB4
:104FF000074B1A784AB9074AFF211170064A4FF049
:10500000804101201160187070470020704700BF78
:10501000B8A7FF1F5EE400E008E100E0F8B5164B1A
:10502000164D1A6842F080721A60154B1A6842F0E9
:1050300001021A60134B2E681C680FE0237A63B1DB
:1050400021682F680B68204698472A68E388D21B9E
:1050500012099A42A28088BFE2806469002CEDD1D7
:10506000064B094A1B689B1B1B091380074A1188C2
:105070008B4288BF1380F8BDFCED00E0041000E017
:10508000001000E0ACA7FF1FD4A7FF1FBAA7FF1FA7
:1050900030B572B609B9026822B9264A00231188D0
:1050A000144611E003790F2BF7D82249098841FAF9
:1050B00003F1C907F1D503F1007303F59063B2EB77
:1050C000431FEAD162B630BD41FA03F212F0010289
:1050D00027D1012505FA03F52943218062B6164937
:1050E00003710C6844F002040C6051F8044C44F065
:1050F000020441F8044C114982240C608B768B77B2
:105100000B76CB7703F1007303F590635B010360CB
:105110001A605A609A60DA601A615A619A61DA61BB
:1051200030BD0133102BCFD162B600220260037173
:1051300030BD00BFD8A7FF1F408004400080004062
:1051400003790F2B10D8094A137072B6084B0279F5
:10515000012101FA02F2198821EA02021A8062B6DC
:105160001023037100230360704700BF1A800040C2
:10517000D8A7FF1F08B5FBF71FFEFCF749F800F0A2
:10518000B5F9FAE7F8B506460C468F18002506E093
:10519000336814F8011B1B68304698472D18BC4231
:1051A000F6D12846F8BDFFFF07B5054B1B88ADF8C3
:1051B0000430036801A95B68022298470EBD00BF56
:1051C00088A40000F0B505468BB022B90368C9B2C7
:1051D0001B6898472CE0012A08BF0A2221B9302217
:1051E0008DF82520212413E02124B1FBF2F002FBED
:1051F0001011C9B2092901D8303100E037310AAFA6
:105200003E1906F8241C014610B1013CE4B2ECE75B
:1052100033B1013C0AAAE4B213192D2203F8242C5D
:105220002B6801AF5B6828463919C4F12202984700
:105230000BB0F0BD002902DA49422D2300E0002323
:105240000A22FFF7BFBF08461146FFF721BD0846F7
:10525000FFF786BDFFF78EBDFFF7EEBCFFF7C4BCBE
:10526000FFF708BD7047FFFF044B00221A711A7345
:10527000034A4FF47A7199601A607047DCA7FF1FE8
:1052800098A4000010B5029C401AE41A4443521A34
:1052900094FBF2F0C01810BD10B50446006803F08E
:1052A00091FA204610BD38B504460D46006801311C
:1052B00003F018FF10B184E82100012038BD4368D5
:1052C0008B4210B5044600D306E0FFF7ECFF20B197
:1052D000A3680BB922681370012010BDF8B504460D
:1052E0000F46154622B9036803B11A7000230BE07C
:1052F0001146FFF7E4FF064640B9206810B103F0FD
:1053000061FA266000236360A36004E0A560206862
:10531000394604F059FA2046F8BD38B50023044652
:1053200003604360836003730D4639B10846FEF79E
:1053300067FD294602462046FFF7D0FF204638BDCC
:1053400081420B4603D009689A68FFF7C7BF7047D0
:10535000002310B504460360436083600373FFF7C6
:10536000EFFF204610BD38B505460C4641B1084652
:10537000FEF746FD214602462846FFF7AFFF00E054
:10538000A960284638BD70B504460E4685685AB1F6
:1053900055192946FFF793FF30B12068A3683146BD
:1053A000C01804F011FAA560204670BD0B460968CC
:1053B0009A68FFF7E8BF38B505460C4639B108468C
:1053C000FEF71EFD214602462846FFF7DCFF284671
:1053D00038BD13B5002304468DF80410012201A93D
:1053E0008DF80530FFF7CFFF20461CBD1FB50446E2
:1053F0000A22084601A9FEF729FD01A8FEF700FDD3
:1054000001A902462046FFF7BEFF204604B010BDAA
:1054100010B50446FFF7DDFF204610BD826808B5D1
:105420000B461AB901B103E0012008BD11B90368A8
:10543000187802E0006804F0D9F8D0F1010038BF14
:10544000002008BD10B58B688468E41AA2420CD80D
:10545000006868B1096851B180181A4604F012FA60
:10546000D0F1010038BF002010BD002010BD08465B
:1054700010BD82688B689A4202D30022FFF7E2BF18
:105480000020704708B582688B689A420CD3006888
:1054900068B1096851B1D31AC01804F0A7F8D0F167
:1054A000010038BF002008BD002008BD084608BD27
:1054B00038B50C469AB191B181688B4202D3002372
:1054C000237038BDCD1A013A0168954228BF1546B0
:1054D000C91820462A4604F02BFA0023635538BD2C
:1054E000006808B103F022B97047FFFF08B50E4B02
:1054F0001A78C2B901221A70FFF7BCFB08B1FFF796
:10550000B1FE00F08BF908B100F0E6FE00F0C4FB3C
:1055100008B100F053FF00F0A9FD08B100F0C0FF92
:10552000014B00221A7008BDECA7FF1F194B1A6827
:1055300042F480621A60184A00231370174A1370ED
:10554000174A1370174A1370174A1370174B40F21B
:1055500013321A604FF451725A60154BC0F3443243
:105560001A70C0F347125A700221042200F01F0083
:1055700098729A70D9745A7588221A743C22DA701B
:105580000C4B40226FF44A711A705B184FF40052B2
:105590001A607047348004406FA8FF1FEEA7FF1FFA
:1055A00078A8FF1F70A8FF1FEDA7FF1F40A00440B1
:1055B00000A006402DE400E0134A937800F00301B8
:1055C00003F0EC030B43410748BF43F01003937013
:1055D00000F00F03042B0C4903D18B7943F04003F7
:1055E0008B715379C20603F0EF03074A48BF43F0BB
:1055F000100353719379800603F0EF0348BF43F023
:1056000010039371704700BF00A006400E4B1B684B
:10561000580510B503D410BDFFF768FF00E00B4C30
:105620002378002BF8D10A4A4FF400511160094A3F
:105630000949D37040F203120A604A60074A1370A6
:10564000074A137010BD00BF34800440EDA7FF1F50
:1056500084E100E000A0064040A004406FA8FF1FC6
:10566000EEA7FF1F38B5094B04461D78002DFCD16D
:1056700020460121FEF7B0FD20462946FEF780FDB9
:10568000034B53F83420034B1A6038BDEDA7FF1FBE
:1056900078A3000074A8FF1F1D4B1B685A052DE955
:1056A000F041074631D51B4B1B680BB101221A7024
:1056B000194B1A4D1C781A4EDFF8688001343F2CC4
:1056C00088BF002414E0FEF77DFB40280CDC337912
:1056D0001B060DD52B7801333F2B88BF002318F80C
:1056E0000320F2712B7003E0FF2801DDFFF7FEFEBF
:1056F0002B78A342E7D00B4B1F550B4B01221A709E
:10570000054B1C70064BBC22DA70BDE8F08100BF6F
:105710003480044074A8FF1F78A8FF1F70A8FF1FE3
:1057200000A00640EFA7FF1FEDA7FF1F2DE9F84FD0
:10573000254B1B6806465805894642D5234B1B68F6
:105740000BB101221A70224DB346AA4632E0214B1A
:105750001C782F7801343F2C88BF0024A74209D041
:105760001BF8012B1C4B1A551C4B01221A70194BAC
:105770001C701FE01A4BBC22DA709846FEF722FB21
:1057800040280FDC98F8043019060FD52B78124A00
:1057900001333F2B88BF0023D25C88F807208AF8AA
:1057A000003003E0FF2801DDFFF7A0FE2B78BB42AD
:1057B000E4D0D5E706EB09039B45C8D3084BBC22D0
:1057C000DA70BDE8F88F00BF3480044074A8FF1F72
:1057D00070A8FF1F78A8FF1FEFA7FF1FEDA7FF1FEF
:1057E00000A0064010B5044C01E0FFF77FFE2378CF
:1057F000002BFAD110BD00BFEDA7FF1F054B064AD5
:105800001B781078834201D33F3000E00138C01A82
:10581000704700BF78A8FF1F70A8FF1F044B1878BF
:10582000044B1B78984238BF4030C01A704700BF05
:105830006FA8FF1FEEA7FF1F084B094A19781378BE
:10584000994207D001333F2B88BF00230549C85C2C
:10585000137070474FF0FF30704700BF6FA8FF1FF5
:10586000EEA7FF1F2FA8FF1F074B1A78074B1B78C7
:105870009A4206D001333F2B88BF0023044AD05CF4
:1058800070474FF0FF3070476FA8FF1FEEA7FF1F54
:105890002FA8FF1F094B1B685B050ED5084BDA7854
:1058A00002F0CB02DA7040225A74DA7842F0340205
:1058B000DA70044B1A78044B1A7070473480044035
:1058C00000A00640EEA7FF1F6FA8FF1F70B52D4B6D
:1058D0001A7912F0300F1DD072B6997D21B9DA799C
:1058E00040225A7462B615E062B6274A27481278F9
:1058F000274D00781C46531C3F2B88BF0023E679B8
:1059000083421CBFEE541A46013911F0FF01F2D157
:105910001D4B1A701B4AD37819465BB2002B1BDA59
:105920001379180618D51B4B1B4C1D781B4B1B7885
:10593000AB4209D001333F2B88BF00231079E05CD4
:10594000D071107D0728F3D9144A13700D4B1A79C2
:10595000120601D57C22DA7001F04003DBB27BB184
:10596000084B1A7902F04002D2B2194642B10C4BF0
:1059700000221A700B4B1B6803B11A703C23CB70CA
:1059800070BD00BF00A006406FA8FF1FEEA7FF1F5D
:105990002FA8FF1F78A8FF1FEFA7FF1F70A8FF1FEA
:1059A000EDA7FF1F74A8FF1F184B1A6842F400628E
:1059B0001A60174A00231370164A1370164A1370A0
:1059C000164A1370164A1370164B40F213321A60BF
:1059D0004FF451725A60144BC0F344321A70C0F342
:1059E00047125A7000F01F000422022198729A7028
:1059F000D9745A7588221A743C22DA700B4B4022F3
:105A00001A700B4B4FF400421A6070473480044008
:105A1000E3A8FF1F7AA8FF1FECA8FF1FE4A8FF1F41
:105A200079A8FF1F0CB0044000B006402FE400E04E
:105A300004E100E0134A937800F0030103F0EC0363
:105A40000B43410748BF43F01003937000F00F036E
:105A5000042B0C4903D18B7943F040038B715379AC
:105A6000C20603F0EF03074A48BF43F01003537127
:105A70009379810603F0EF0348BF43F0100393715D
:105A8000704700BF00B006400E4B1B68180510B5EC
:105A900003D410BDFFF72AFD00E00B4C2378002B48
:105AA000F8D10A4A4FF400411160094A0949D370FC
:105AB00040F203120A604A60074A1370074A1370E3
:105AC00010BD00BF3480044079A8FF1F84E100E0CE
:105AD00000B006400CB00440E3A8FF1F7AA8FF1FE7
:105AE00038B5094B04461D78002DFCD12046012114
:105AF000FEF772FB20462946FEF742FB034B53F8A4
:105B00003420034B1A6038BD79A8FF1F78A300002A
:105B1000E8A8FF1F1D4B1B681A052DE9F041074639
:105B200031D51B4B1B680BB101221A70194B1A4D52
:105B30001C781A4EDFF868800134272C88BF0024B7
:105B400014E0FEF73FF940280CDC33791B060DD535
:105B50002B780133272B88BF002318F80320F2711C
:105B60002B7003E0FF2801DDFFF7C0FC2B78A34278
:105B7000E7D00B4B1F550B4B01221A70054B1C70C5
:105B8000064BBC22DA70BDE8F08100BF34800440CF
:105B9000E8A8FF1FECA8FF1FE4A8FF1F00B0064005
:105BA0007BA8FF1F79A8FF1F2DE9F84F254B1B6825
:105BB00006461805894642D5234B1B680BB10122C6
:105BC0001A70224DB346AA4632E0214B1C782F783A
:105BD0000134272C88BF0024A74209D01BF8012BD1
:105BE0001C4B1A551C4B01221A70194B1C701FE0DC
:105BF0001A4BBC22DA709846FEF7E4F840280FDC16
:105C000098F8043019060FD52B78124A0133272B48
:105C100088BF0023D25C88F807208AF8003003E0B0
:105C2000FF2801DDFFF762FC2B78BB42E4D0D5E70B
:105C300006EB09039B45C8D3084BBC22DA70BDE8CC
:105C4000F88F00BF34800440E8A8FF1FE4A8FF1FBE
:105C5000ECA8FF1F7BA8FF1F79A8FF1F00B006401C
:105C600010B5044C01E0FFF741FC2378002BFAD17A
:105C700010BD00BF79A8FF1F054B064A1B7810789E
:105C8000834201D3273000E00138C01A704700BFBB
:105C9000ECA8FF1FE4A8FF1F044B1878044B1B78E7
:105CA000984238BF4030C01A704700BFE3A8FF1FBA
:105CB0007AA8FF1F084B094A19781378994207D030
:105CC00001333F2B88BF00230549C85C1370704720
:105CD0004FF0FF30704700BFE3A8FF1F7AA8FF1FF7
:105CE000A3A8FF1F074B1A78074B1B789A4206D0D0
:105CF00001333F2B88BF0023044AD05C70474FF02C
:105D0000FF307047E3A8FF1F7AA8FF1FA3A8FF1F5B
:105D1000094B1B681B050ED5084BDA7802F0CB0245
:105D2000DA7040225A74DA7842F03402DA70044BA6
:105D30001A78044B1A7070473480044000B0064053
:105D40007AA8FF1FE3A8FF1F70B52D4B1A7912F038
:105D5000300F1DD072B6997D21B9DA7940225A747C
:105D600062B615E062B6274A27481278274D0078B8
:105D70001C46531C3F2B88BF0023E67983421CBF7F
:105D8000EE541A46013911F0FF01F2D11D4B1A7081
:105D90001B4AD37819465BB2002B1BDA137918061D
:105DA00018D51B4B1B4C1D781B4B1B78AB4209D0E5
:105DB0000133272B88BF00231079E05CD071107D60
:105DC0000728F3D9144A13700D4B1A79120601D51E
:105DD0007C22DA7001F04003DBB27BB1084B1A7908
:105DE00002F04002D2B2194642B10C4B00221A70A6
:105DF0000B4B1B6803B11A703C23CB7070BD00BF06
:105E000000B00640E3A8FF1F7AA8FF1FA3A8FF1F4A
:105E1000ECA8FF1F7BA8FF1FE4A8FF1F79A8FF1FA6
:105E2000E8A8FF1F174B1A6842F480521A60164AFE
:105E300000231370154A1370154A1370154A137016
:105E4000154A1370154A40F2133111604FF4517125
:105E50005160134AC0F344311170C0F3471100F090
:105E60001F0051709072937013742C23D3700D4BDC
:105E700040226FF44B711A705B184FF400321A60B5
:105E8000704700BF3480044057A9FF1FEEA8FF1FD2
:105E900060A9FF1F58A9FF1FEDA8FF1F08C00440FD
:105EA00000C0064031E400E0134A937800F003019B
:105EB00003F0EC030B43410748BF43F0100393701A
:105EC00000F00F03042B0C4903D18B7943F04003FE
:105ED0008B715379C20603F0EF03074A48BF43F0C2
:105EE000100353719379800603F0EF0348BF43F02A
:105EF00010039371704700BF00C006400E4B1B6833
:105F0000D80410B503D410BDFFF7F0FA00E00B4C35
:105F10002378002BF8D10A4A4FF400311160094A66
:105F20000949D37040F203120A604A60074A1370AD
:105F3000074A137010BD00BF34800440EDA8FF1F56
:105F400084E100E000C0064008C0044057A9FF1FDC
:105F5000EEA8FF1F38B5094B04461D78002DFCD173
:105F600020460121FEF738F920462946FEF708F9B8
:105F7000034B53F83420034B1A6038BDEDA8FF1FC4
:105F800078A300005CA9FF1F1D4B1B68DA042DE9F4
:105F9000F041074631D51B4B1B680BB101221A702B
:105FA000194B1A4D1C781A4EDFF868800134272CE3
:105FB00088BF002414E0FDF705FF40280CDC33798E
:105FC0001B060DD52B780133272B88BF002318F82B
:105FD0000320F2712B7003E0FF2801DDFFF786FA42
:105FE0002B78A342E7D00B4B1F550B4B01221A70A5
:105FF000054B1C70064BAC22DA70BDE8F08100BF87
:10600000348004405CA9FF1F60A9FF1F58A9FF1F2F
:1060100000C00640EFA8FF1FEDA8FF1F38B54518C8
:10602000044603E014F8010BFFF7AEFFAC42F9D1D0
:1060300038BDFFFF10B5044C01E0FFF757FA237895
:10604000002BFAD110BD00BFEDA8FF1F054B064A7B
:106050001B781078834201D3273000E00138C01A42
:10606000704700BF60A9FF1F58A9FF1F044B187895
:10607000044B1B78984238BF4030C01A704700BFAD
:1060800057A9FF1FEEA8FF1F084B094A197813787C
:10609000994207D001333F2B88BF00230549C85CD4
:1060A000137070474FF0FF30704700BF57A9FF1FB4
:1060B000EEA8FF1F17A9FF1F074B1A78074B1B7885
:1060C0009A4206D001333F2B88BF0023044AD05C9C
:1060D00070474FF0FF30704757A9FF1FEEA8FF1F12
:1060E00017A9FF1F024B1A78024B1A70704700BFA6
:1060F000EEA8FF1F57A9FF1F10B5214B1A7902F018
:106100002002D2B26AB11F4AD8791F4913780978A0
:1061100001333F2B88BF00238B4202D01B49C85458
:106120001370174AD37818465BB2002B13DA137931
:10613000190610D5164B17491C780B789C4202D1D2
:106140006C23D37007E00133272B88BF0023124C48
:10615000E45CD4710B7000F04003DBB27BB1084B00
:106160001A7902F04002D2B2194642B10B4B00221A
:106170001A700B4B1B6803B11A702C23CB7010BD27
:1061800000C0064057A9FF1FEEA8FF1F17A9FF1F59
:1061900060A9FF1F58A9FF1FEFA8FF1FEDA8FF1F51
:1061A0005CA9FF1F1FB572B6154B70221A70154AF5
:1061B000412111700F2102F8011C80221A701A78F7
:1061C0001206FCD5104B186862B6104B984201D8E5
:1061D0000A23584301A90A22FDF71AFE0C4800239E
:1061E00001AA9A5C2AB100EB430101330A2B4A80D1
:1061F000F6D10133064A5B00137005B000BD00BF45
:106200000000024007000240080002407F9698000C
:106210003890FF1F08B50368C9B21B68984708BDCE
:1062200008B50368C9B21B68984708BD08B503687C
:10623000C9B21B68984708BD08B50368C9B21B6896
:10624000984708BD084608B5FFF726FA012008BDA3
:10625000084608B5FFF720FA012008BD38B5084602
:106260000D46FDF7CDFD044621462846FFF75EFAB0
:10627000204638BD10B5084614461146FFF756FAB9
:10628000204610BDFFF7BABAFFF704BBFFF7AABA62
:10629000FFF7D2BAFFF7E8BAFFF7C0BA0846FFF730
:1062A000E1B9FFF7B3B9480800F1376000F5D8301D
:1062B000B0FBF1F0FFF73AB9480800F1376010B5CC
:1062C00000F5D830B0FBF1F01446FFF72FF9204667
:1062D000BDE81040FFF770B97047FFFF044B002284
:1062E0001A711A73034A4FF47A7199601A607047F1
:1062F00064A9FF1F10A5000008B50368C9B21B6898
:10630000984708BD08B50368C9B21B68984708BD1F
:1063100008B50368C9B21B68984708BD08B503688B
:10632000C9B21B68984708BD084608B5FFF7F2FBDD
:10633000012008BD084608B5FFF7ECFB012008BDA9
:1063400038B508460D46FDF75BFD04462146284654
:10635000FFF72AFC204638BD10B508461446114602
:10636000FFF722FC204610BDFFF786BCFFF7D0BC2C
:10637000FFF776BCFFF79EBCFFF7B4BCFFF78CBC01
:106380000846FFF7ADBBFFF77FBB480800F1376059
:1063900000F5D830B0FBF1F0FFF706BB480800F17C
:1063A000376010B500F5D830B0FBF1F01446FFF7B8
:1063B000FBFA2046BDE81040FFF73CBB7047FFFFEB
:1063C000044B00221A711A73034A4FF47A719960D0
:1063D0001A60704774A9FF1F60A5000008B5036824
:1063E000C9B21B68984708BD08B50368C9B21B68E5
:1063F000984708BD08B50368C9B21B68984708BD2F
:1064000008B50368C9B21B68984708BD084608B5B7
:10641000FFF7BAFD012008BD084608B5FFF7B4FD37
:10642000012008BD38B508460D46FDF7E9FC0446D5
:1064300021462846FFF7F2FD204638BD10B5084634
:1064400014461146FFF7EAFD204610BDFFF7FEBDDA
:10645000FFF748BEFFF7EEBDFFF716BEFFF72CBEF5
:10646000FFF704BE0846FFF775BDFFF747BD4808B4
:1064700000F1B76000F55840B0FBF1F0FFF7D2BC77
:10648000480800F1B76010B500F55840B0FBF1F0D6
:106490001446FFF7C7FC2046BDE81040FFF704BDD7
:1064A0007047FFFF044B00221A711A73034A4FF41E
:1064B0007A7199601A60704784A9FF1FB0A5000027
:1064C0002DE9F04F8BB01F4680468946164600F0F6
:1064D00093F949F24E0BC1F6FF7B9BF90030013373
:1064E00004460D4604D03046394600F0F5FF20B989
:1064F000204629460BB0BDE8F08F4046494600F0E3
:10650000EBFF824620BB304639460022002301F0D3
:1065100059FD0028ECD09BF900104AF2F8530122F3
:10652000C0F200038DE80C0000220023B1F1FF3F10
:1065300018BF0229C3F6F073CDF820A0CDE9028977
:10654000CDE90467CDE906232DD1DDE90645CFE786
:10655000404649460022002301F034FD00282FD098
:10656000304639460022002301F02CFD002861D07E
:106570009BF900204AF2F853C0F2000301210020E9
:106580008DE80A00CDE90289002300210893CDE9B6
:106590000467CDE9060132B100230022C3F6F0738F
:1065A000CDE90623D1E7684600F0BEFF002870D091
:1065B000089B002BC9D002F0CBF8089B0360C4E70E
:1065C0002046294600F082FF8246002866D02046F9
:1065D00029460022002301F0F5FC002888D040461F
:1065E000494600F073FF002882D03046394600F05B
:1065F0006DFF00283FF47CAF9BF900204AF2F8536E
:106600000421C0F2000300208DE80A0000230021CD
:10661000022A0893CDE90289CDE90467CDE9060194
:1066200069D0684600F080FF002864D0089B002BEA
:106630008BD0C0E73046394600F048FF00283FF4D1
:1066400057AF304639460022002301F0C5FC002830
:106650003FF44EAF9BF800104AF2F853C0F200032B
:106660000122CDE902898DE80C000023CDE9046701
:10667000002208930023002936D1CDE9062368467D
:1066800000F052FF0028D1D102F062F8212303600C
:10669000CCE702F05DF82123036089E740464946D4
:1066A00000F014FF002892D03046394600F00EFF6B
:1066B00000288CD02046294600F00EFF00BB9BF836
:1066C00000404AF2F853C0F2000301220890002172
:1066D0008DE80C000020CDE90289CDE90467002C8B
:1066E00063D1CDE90601CAE70229CFF6F073CDE9FF
:1066F0000623C9D0C3E702F02BF82223036095E7F5
:106700009BF900104AF2F8520320C0F20002CDF8C3
:1067100020A08DE805004046CDE90289CDE9046757
:10672000E9B94FF6FF754946002200234FF0604457
:10673000C4F2EF75CDE9064501F04EFC00283ED1CC
:106740009BF90030022B05D0684600F0EDFE0028D2
:106750007FF42EAF01F0FCFF2223036028E7002521
:106760004946002200230024C7F6F075CDE906450E
:1067700001F032FC0028E3D000230022C3F6E073CE
:106780003046394601F0B6F904460D4600F0D4FE15
:1067900022462B4601F016FC0028D1D1002300220E
:1067A000CFF6F073CDE90623CAE702460B4601F0A7
:1067B000CBFA022CCDE906013FF466AF5FE7002378
:1067C0000022C3F6E0733046394601F093F90446DF
:1067D0000D4600F0B1FE22462B4601F0F3FB0028E7
:1067E000AED14FF6FF734FF06042CCF2EF73CDE9BC
:1067F0000623A5E7FFFFFFFF2DE9F04F91B023F03F
:1068000000478B460D46049157EA020191468246A5
:106810001E4604469446804600F08E8000212BF0F0
:106820000040C7F6F0710290884211DD029901F133
:10683000404909F5801959EA080840F0828000268D
:10684000C146C3F6F0764846314611B0BDE8F08F38
:1068500014BF002001200690BAF1000F0CBF0020E9
:1068600000F001000028E1D18F42DFDC14BF0020DE
:106870000120002A0CBF002100F001010029D5D120
:10688000049A5C461D46002A64DB0E91BCF1000FA1
:1068900014D1002840F082800023C3F6F0739F4299
:1068A00000F0B880B5F1804F04BF504659463CD047
:1068B0000023C3F6E0739D4200F0C0835046594662
:1068C00000F000FE8C46B8F1000F0BD1069B029938
:1068D000002908BF43F00103002B76D1C3F6F07303
:1068E000994272D0049B0E994FEAD37808F1FF3891
:1068F00051EA080100F089800023C4F2E0139F42AE
:1069000040F3A6800023C4F2F0339F4240F330846A
:106910004FF6FF73029AC3F6EF739A4240F39E83D9
:10692000002D4EDD48A1D1E9000102460B4601F0E1
:10693000E1F881460E4686E700268946C3F6F076E2
:1069400081E74AF23060C0F2000011B0BDE8F04FBC
:1069500000F0ECBD4FF6FF73C4F23F339F426ADC98
:106960004FF6FF73C3F6EF739F428EDD3B1540F287
:106970001342934240F38B84C3F5866303332CFAAE
:1069800003F202FA03F3634502BF02F00103C3F10D
:1069900002030E933FF47AAF002176E7029A02F1E8
:1069A000404303F5801353EA080300F051834FF688
:1069B000FF73C3F6EF739A4240F3B283002DBFF624
:1069C00042AF4FF000094E463DE7002DA8BF664696
:1069D000C0F24284002CA8BF8146BFF634AF029AB1
:1069E0000E9902F1404303F58013194340F05F8490
:1069F000804602463346314600F0C8FE02460B464A
:106A000001F0A2F981460E461DE75046594652460E
:106A10005B46F1E7002DA4BFD1465E46BFF613AF3B
:106A2000002152460020C3F6F0715B4601F08CF95C
:106A300081460E4607E702230E93BCF1000F3FF498
:106A400028AF3BE7AFF300809C7500883CE4377EBD
:106A5000029B0021B3F5801F0BDA00236146002260
:106A6000C4F2403301F046F88C466FF03401CDF8A3
:106A700008C0029A002522F07F43141549F68E02C1
:106A800023F47003C0F20302934243F07F57A4F251
:106A9000FF340C440F9447F440142F460FDD4BF2A3
:106AA00079620127C0F20B024FF48025934206DD84
:106AB00000250F9BA4F580142F4601330F934AF253
:106AC00000610246C0F20001234601EBC707CDE991
:106AD0000823D7E90001CDE90A0110462146DDE986
:106AE0000A2300F053FEDDE90A2382468B46DDE9E6
:106AF000080100F04DFE0B4600210246C3F6F0717E
:106B0000002001F021F9CDE90C015046DDE90C230C
:106B1000594600F0EFFFCDE906016110DDE90623DB
:106B200041F00051002001F50021CDE904236B184C
:106B300004900022DDE9040114461D46CDE902015E
:106B400000F0D8FF02460B465046594600F01EFEA4
:106B5000DDE90A2382468B462046294600F016FED0
:106B600002460B46DDE9080100F010FE02460B4626
:106B7000DDE9020100F0BEFF02460B4650465946D1
:106B800000F004FEDDE90C2300F0B4FF82468B46E2
:106B9000DDE9060102460B4600F0ACFF02460B465B
:106BA00004460D4600F0A6FFA3A3D3E90023CDE9D8
:106BB00008012046294600F09DFFA1A3D3E9002348
:106BC00000F0E6FD22462B4600F094FF9EA3D3E999
:106BD000002300F0DDFD22462B4600F08BFF9CA336
:106BE000D3E9002300F0D4FD22462B4600F082FFBB
:106BF00099A3D3E9002300F0CBFD22462B4600F0F9
:106C000079FF97A3D3E9002300F0C2FD02460B46AB
:106C1000DDE9080100F06EFFDDE9062304460D46BC
:106C2000DDE9020100F0B4FD52465B4600F062FF70
:106C300022462B4600F0ACFDCDE90801DDE902015A
:106C400002460B4600F056FF00220023C4F2080360
:106C5000CDE90A0100F09CFDDDE9082300F098FD74
:106C60000D4604992B460C46DDE90201224600F050
:106C700041FF22462B46CDE902015046594600F01D
:106C800039FF00230022C4F2080382468B462046C7
:106C9000294600F07BFDDDE90A2300F077FD02467E
:106CA0000B46DDE9080100F071FDDDE9062300F087
:106CB00021FF02460B465046594600F069FD8246C8
:106CC0008B4652465B46DDE9020100F061FD049A05
:106CD000104665A3D3E9002304460D4600F00AFFE1
:106CE00063A3D3E90023CDE906012046294600F03D
:106CF00001FFDDE90223CDE908012046294600F025
:106D000045FD02460B465046594600F03FFD5AA34A
:106D1000D3E9002300F0EEFE02460B46DDE9080150
:106D200000F036FDD7E9042300F032FD82460F98CB
:106D30008B4600F079FE52465B4604460D46D7E985
:106D40000801CDE90201DDE9060100F021FDDDE9E0
:106D5000022300F01DFD22462B4600F019FD049A87
:106D60002B461046224604460D4600F00FFDDDE995
:106D7000022300F00BFDDDE9062300F007FD0246CB
:106D80000B465046594600F001FD82468B460E9850
:106D9000431E53EA080340F0BC8100230022CBF6D7
:106DA000F073CDE904233346002231464846CDE94D
:106DB000022300F0EBFC22462B4600F09BFE5246DD
:106DC0005B46CDE906013146484600F093FE024697
:106DD0000B46DDE9060100F0DBFC22462B4682462D
:106DE0008B46DDE9020100F085FE04460D46504663
:106DF000594622462B4600F0CBFC4FF6FF7CC4F2EE
:106E00008F0C614506460F46884640F32B8101F101
:106E10003F4303F5E003034340F0298218A3D3E97D
:106E200000235046594627F0004900F0B1FC2246A5
:106E30002B46CDE9020127E0EF4E454A287ECA3FA6
:106E400065DBC9934A86CD3F01411DA96074D13FDE
:106E50004D268F515555D53FFFAB6FDBB66DDB3FF0
:106E6000033333333333E33F000000E009C7EE3F21
:106E7000F5015B14E02F3EBEFD033ADC09C7EE3F8F
:106E8000FE822B654715973C3046394600F07EFC64
:106E900002460B46DDE9020101F0BCF8002840F093
:106EA000E6810023C3F6E0739945DCBF4FF0000C88
:106EB000CDF808C000F3F48000269DA3D3E9002399
:106EC00030463946CDF804C000F014FE22462B4669
:106ED000804689463046394600F058FC02460B464B
:106EE0005046594600F052FC93A3D3E9002300F02A
:106EF00001FE93A3D3E9002304460D4630463946EC
:106F000000F0F8FD02460B462046294600F040FC02
:106F100004460D4622462B464046494600F038FCC2
:106F200042464B4682468B4600F030FC02460B46FA
:106F30002046294600F02AFC52465B468046894698
:106F40005046594600F0D6FD7FA3D3E900230446FE
:106F50000D4600F0CFFD7EA3D3E9002300F016FC20
:106F600022462B4600F0C6FD7BA3D3E9002300F0A8
:106F70000FFC22462B4600F0BDFD79A3D3E9002388
:106F800000F004FC22462B4600F0B4FD76A3D3E9C2
:106F9000002300F0FDFB22462B4600F0ABFD02462D
:106FA0000B465046594600F0F1FB04460D4622467A
:106FB0002B465046594600F09DFD00224FF080437D
:106FC00006460F462046294600F0E0FB02460B46E7
:106FD0003046394600F0B8FE42464B4604460D4660
:106FE0005046594600F086FD42464B4600F0D0FB25
:106FF00002460B462046294600F0C8FB52465B4637
:1070000000F0C4FB0B4600210246C3F6F0710020DD
:1070100000F0BCFBDDF804C00CEB01040B46B4F53A
:10702000801F02460D46A8BF2346C0F25E81DDE9FF
:10703000040100F05FFD81460E4604E4002CFFF6DB
:107040003DAC5046594611B0BDE8F04F00F074B960
:1070500000269946C3F6F076FFF7F5BB002DBFF684
:10706000B0AC5FE44CF6FF3321F00049C4F290036A
:1070700099457FF716AF4FF45053C3F66F73CB1893
:10708000034340F01A8122462B4600F07FFB024664
:107090000B465046594600F0A9FF002840F00D81EC
:1070A0004FEA29534FF48011A3F2FE334FF6FF76D7
:1070B00041FA03F1C0F20F064144002221F07F475C
:1070C000C1F30A5027F47007A0F2FF3E47F480177F
:1070D000C0F58260B8F1000F46FA0EF600F1030C1D
:1070E00021EA060347FA0CFCCDF808C0C0F2F9808B
:1070F0002046294600F04AFB04460D4622465046EB
:1071000059462B4600F044FB029A4FEA025C0F46B8
:10711000D2E600210020C3F6F071CDE9040142E679
:10712000002DBFF64EAC06F10046FFF78CBB00BF4A
:1071300000000000432EE63FEF39FAFE422EE63F04
:10714000396CA80C615C20BED0A4BE726937663E63
:10715000F16BD2C541BDBB3E2CDE25AF6A56113F57
:1071600093BDBE166CC1663F3E5555555555C53F3E
:107170004FF6FE730299C3F6EF7399427FF76EAF35
:107180000023029AC3F6F0739A423FF7C9AB00237B
:1071900061460022C3F6F07300F0F8FA5AA3D3E96F
:1071A000002304460D4600F0A5FC59A3D3E90023B3
:1071B00082468B462046294600F09CFC22462B4600
:1071C000CDE902012046294600F094FC002300226C
:1071D000C3F6D073CDE904012046294600F08AFCAD
:1071E00002460B464CA1D1E9000100F0CFFA22463D
:1071F0002B4600F07FFC0B4600210246C3F6E071EF
:10720000002000F0C3FA02460B46DDE9040100F05D
:1072100071FC43A3D3E9002300F06CFC02460B464B
:10722000DDE9020100F0B2FACDE902015046DDE9E4
:107230000223594600F0ACFA52465B460020044651
:107240000D4600F0A3FA02460B46DDE9020100F00C
:107250009DFA82468B469AE500210246C3F6F071FC
:107260000020634600F070FD0E46FFF7B3BB2EA36F
:10727000D3E90023DDE9040100F03CFC2AA3D3E9B3
:10728000002300F037FC81460E46FFF7DCBABCF164
:10729000000F22D1C3F58263DA1C47FA02F303FA26
:1072A00002F2BA4227D000230E93FFF7F2BA0E9AE9
:1072B0008146012A7FF4C7AA35E71DA3D3E900233D
:1072C000DDE9040100F016FC19A3D3E9002300F066
:1072D00011FC81460E46FFF7B6BA00230E93FFF766
:1072E000EDBA61464942029102E7029A00F0BCF908
:1072F00002460B469BE603F00103C3F102030E9323
:10730000FFF7C7BAAFF30080000000604715F73FF2
:1073100044DF5DF80BAE543E555555555555D53F98
:10732000FE822B654715F73F9C7500883CE4377E4D
:1073300059F3F8C21F6EA5012DE9F8430027B9469D
:10734000C7F6F077C7F6F0790F404F4504460D4673
:1073500002460B460E46804600F09980002977DDF4
:107360000F1500F0828026F07F43A7F2FF3723F449
:107370007003FA0743F4801344BF4FEAD8724FEA10
:1073800048084FF0000C48BF02EB430360464FEA49
:10739000D8727F1002EB430316244FEA48024FF4E1
:1073A00000114518D60F9D424FEA4202DEBFC5EBE1
:1073B000030368188C444908013C06EB4303F0D1F1
:1073C0002026A0464FF000410EE081461B1A954250
:1073D00088BF013B521B64184846D50F490852002C
:1073E000013E05EB430315D0984201EB080503DB92
:1073F000954298BF8342F0D105F0004905EB0108A2
:10740000B9F1004FE1D1B8F1000FA8BF00F10109B7
:10741000DCDADAE7134312D166084FEA6C031CF09A
:10742000010F03F17F5318BF46F0004603F5001328
:10743000344603EB075520462946BDE8F883631C14
:1074400008BF0CF1010CE8D004F001031C19E3E7BC
:1074500021F000460643EED041BB0F464FEAD82646
:10746000153F4FEA4858002EF8D016F4801319D172
:1074700076000133F102FBD5C3F10101C3F1200213
:1074800028FA02F27F18164308FA03F86BE700F0B7
:1074900031FB02460B462046294600F079F90446A6
:1074A0000D46C8E7202201210023E9E702460B46EA
:1074B00000F06CF902460B4600F046FC04460D460F
:1074C000B9E700BF21F00041704700BF41F0004123
:1074D00001F58010C00F704750EA010201D102206F
:1074E0007047D0F1010238BF0022B1F1004F08BF50
:1074F0000028F4D021F000434FF6FF71A3F580106F
:10750000C7F6DF71884201D804207047B3F5801FA9
:1075100001D2032070470020C7F6F070834214BFE9
:10752000002002F001007047002070470021002079
:10753000C7F6F871704700BFC1F30A5C02462DE937
:10754000F041ACF2FF36CD0F132E82B00B4604464D
:107550000F4688463ADC002E56DB4FF6FF71C0F22C
:107560000F0141FA06F101EA0300104329D049084E
:107570000B4053EA02040CD04FF4802327EA0108A1
:10758000132E0CBF4FF00044002443FA06F648EADD
:1075900006084AF238612246C0F20001434601EB78
:1075A000C505D5E900452046294600F0F1F82246F8
:1075B0002B46CDE90001DDE9000100F0E7F80246C5
:1075C0000B461046194602B0BDE8F081332E07DDA8
:1075D000B6F5806FF5D100F0DBF802460B46F0E718
:1075E0004FF0FF31ACF2134C21FA0CF10142E8D01C
:1075F000490801421FBF4FF0804320EA010443FACB
:107600000CFC44EA0C04C4E721F000410143D8D04B
:1076100023F07F404AF2386120F47000C0F200018C
:1076200040EA020401EBC50160424FEA534E0443B5
:10763000D1E90067240B304604F40024394644EABB
:107640004E4300F0A5F832463B46CDE90001DDE9A6
:10765000000100F09BF80F4621F00041064602466B
:1076600041EAC573ADE700BFC1F30A532DE9F0410C
:1076700004460D46904606460F46C3B921F0004C1D
:107680005CEA000C29D000230022C4F2503300F041
:1076900031FA43F6B043CFF6FF73984504460D46E2
:1076A00006460F462BDBC1F30A53363B05E040F29A
:1076B000FF72934218BF094636D0434440F2FE722F
:1076C0009342C4BF22462B4621DC002B09DD21F06A
:1076D000FF4121F4E00141EA035520462946BDE877
:1076E000F08113F1350F26DA4CF2503322469845DB
:1076F0002B460CDC1AA1D1E9000100F039F818A3DF
:10770000D3E9002300F0F6F904460D46E5E716A19B
:10771000D1E9000100F02CF813A3D3E9002300F015
:10772000E9F904460D46D8E72B46024600F030F84A
:1077300004460D46D1E7363321F0FF4121F4E00144
:10774000204641EA0355002329460022C3F6904310
:1077500000F0D0F904460D46BFE700BFAFF300804C
:1077600059F3F8C21F6EA5019C7500883CE4377E72
:1077700010B421F0004203F0004444EA020110BCBE
:10778000704700BF81F0004102E000BF83F000437A
:1077900030B54FEA41044FEA430594EA050F08BFAC
:1077A00090EA020F1FBF54EA000C55EA020C7FEA70
:1077B000645C7FEA655C00F0E2804FEA5454D4EBED
:1077C0005555B8BF6D420CDD2C4480EA020281EAB7
:1077D000030382EA000083EA010180EA020281EAEF
:1077E0000303362D88BF30BD11F0004F4FEA013141
:1077F0004FF4801C4CEA113102D0404261EB410150
:1078000013F0004F4FEA03334CEA133302D05242D5
:1078100063EB430394EA050F00F0A780A4F1010491
:10782000D5F1200E0DDB02FA0EFC22FA05F28018CB
:1078300041F1000103FA0EF2801843FA05F35941B1
:107840000EE0A5F120050EF1200E012A03FA0EFC30
:1078500028BF4CF0020C43FA05F3C01851EBE3715A
:1078600001F0004507D54FF0000EDCF1000C7EEB77
:1078700000006EEB0101B1F5801F1BD3B1F5001FB5
:107880000CD349085FEA30004FEA3C0C04F10104D4
:107890004FEA445212F5800F80F09A80BCF1004FFD
:1078A00008BF5FEA500C50F1000041EB045141EA7F
:1078B000050130BD5FEA4C0C404141EB010111F480
:1078C000801FA4F10104E9D191F0000F04BF01462B
:1078D0000020B1FA81F308BF2033A3F10B03B3F109
:1078E00020020CDA0C3208DD02F1140CC2F10C0299
:1078F00001FA0CF021FA02F10CE002F11402D8BFF7
:10790000C2F1200C01FA02F120FA0CFCDCBF41EAC2
:107910000C019040E41AA2BF01EB0451294330BD91
:107920006FEA04041F3C1CDA0C340EDC04F114046E
:10793000C4F1200220FA04F001FA02F340EA030045
:1079400021FA04F345EA030130BDC4F10C04C4F18B
:10795000200220FA02F001FA04F340EA030029466B
:1079600030BD21FA04F0294630BD94F0000F83F4B5
:10797000801306BF81F480110134013D4EE77FEA98
:10798000645C18BF7FEA655C29D094EA050F08BFE4
:1079900090EA020F05D054EA000C04BF19461046C5
:1079A00030BD91EA030F1EBF0021002030BD5FEA09
:1079B000545C05D14000494128BF41F0004130BD31
:1079C00014F580043CBF01F5801130BD01F0004585
:1079D00045F0FE4141F470014FF0000030BD7FEAF8
:1079E000645C1ABF194610467FEA655C1CBF0B46F3
:1079F000024650EA013406BF52EA033591EA030F0A
:107A000041F4002130BD00BF90F0000F04BF002101
:107A1000704730B54FF4806404F132044FF0000534
:107A20004FF0000150E700BF90F0000F04BF0021AD
:107A3000704730B54FF4806404F1320410F0004513
:107A400048BF40424FF000013EE700BF42004FEA0E
:107A5000E2014FEA31014FEA02701FBF12F07F438B
:107A600093F07F4F81F06051704792F0000F14BF88
:107A700093F07F4F704730B54FF4607401F00045CC
:107A800021F0004120E700BF50EA010208BF704723
:107A900030B54FF000050AE050EA010208BF704718
:107AA00030B511F0004502D5404261EB41014FF481
:107AB000806404F132045FEA915C3FF4DCAE4FF085
:107AC00003025FEADC0C18BF03325FEADC0C18BF6C
:107AD000033202EBDC02C2F1200300FA03FC20FABD
:107AE00002F001FA03FE40EA0E0021FA02F114440A
:107AF000C1E600BF70B54FF0FF0C4CF4E06C1CEA1F
:107B000011541DBF1CEA135594EA0C0F95EA0C0F93
:107B100000F0DEF82C4481EA030621EA4C5123EA06
:107B20004C5350EA013518BF52EA033541F4801135
:107B300043F4801338D0A0FB02CE4FF00005E1FBE8
:107B400002E506F00042E0FB03E54FF00006E1FB32
:107B500003569CF0000F18BF4EF0010EA4F1FF0475
:107B6000B6F5007F64F5407404D25FEA4E0E6D41B5
:107B700046EB060642EAC62141EA55514FEAC520C6
:107B800040EA5E504FEACE2EB4F1FD0C88BFBCF542
:107B9000E06F1ED8BEF1004F08BF5FEA500E50F1F3
:107BA000000041EB045170BD06F0004646EA0101B9
:107BB00040EA020081EA0301B4EB5C04C2BFD4EBEB
:107BC0000C0541EA045170BD41F480114FF0000EE4
:107BD000013C00F3AB8014F1360FDEBF002001F052
:107BE000004170BDC4F10004203C35DA0C341BDCCC
:107BF00004F11404C4F1200500FA05F320FA04F09E
:107C000001FA05F240EA020001F0004221F00041D1
:107C100010EBD37021FA04F642EB06015EEA430E44
:107C200008BF20EAD37070BDC4F10C04C4F1200574
:107C300000FA04F320FA05F001FA04F240EA020027
:107C400001F0004110EBD37041F100015EEA430EF8
:107C500008BF20EAD37070BDC4F1200500FA05F218
:107C60004EEA020E20FA04F301FA05F243EA020397
:107C700021FA04F001F0004121FA04F220EA0200A6
:107C800000EBD3705EEA430E08BF20EAD37070BDEC
:107C900094F0000F0FD101F00046400041EB0101CC
:107CA00011F4801F08BF013CF7D041EA060195F0AE
:107CB000000F18BF704703F00046520043EB030368
:107CC00013F4801F08BF013DF7D043EA0603704755
:107CD00094EA0C0F0CEA135518BF95EA0C0F0CD060
:107CE00050EA410618BF52EA4306D1D181EA0301A6
:107CF00001F000414FF0000070BD50EA410606BFA0
:107D00001046194652EA430619D094EA0C0F02D1E4
:107D100050EA013613D195EA0C0F05D152EA033629
:107D20001CBF104619460AD181EA030101F0004147
:107D300041F0FE4141F470014FF0000070BD41F090
:107D4000FE4141F4780170BD70B54FF0FF0C4CF46A
:107D5000E06C1CEA11541DBF1CEA135594EA0C0F89
:107D600095EA0C0F00F0A7F8A4EB050481EA030ED6
:107D700052EA03354FEA013100F088804FEA0333BD
:107D80004FF0805545EA131343EA12634FEA02228B
:107D900045EA111545EA10654FEA00260EF000414C
:107DA0009D4208BF964244F1FD0404F5407402D29E
:107DB0005B084FEA3202B61A65EB03055B084FEA2F
:107DC00032024FF480104FF4002CB6EB020E75EB2C
:107DD000030E22BFB61A754640EA0C005B084FEA54
:107DE0003202B6EB020E75EB030E22BFB61A7546D1
:107DF00040EA5C005B084FEA3202B6EB020E75EB1C
:107E0000030E22BFB61A754640EA9C005B084FEA93
:107E10003202B6EB020E75EB030E22BFB61A7546A0
:107E200040EADC0055EA060E18D04FEA051545EA8F
:107E300016754FEA06164FEAC30343EA52734FEA38
:107E4000C2025FEA1C1CC0D111F4801F0BD141EAB1
:107E500000014FF000004FF0004CB6E711F4801F16
:107E600004BF01430020B4F1FD0C88BFBCF5E06FF6
:107E70003FF6AFAEB5EB030C04BFB6EB020C5FEA06
:107E8000500C50F1000041EB045170BD0EF0004E5B
:107E90004EEA113114EB5C04C2BFD4EB0C0541EA8D
:107EA000045170BD41F480114FF0000E013C90E68A
:107EB00045EA060E8DE60CEA135594EA0C0F08BF4E
:107EC00095EA0C0F3FF43BAF94EA0C0F0AD150EA4D
:107ED00001347FF434AF95EA0C0F7FF425AF1046E0
:107EE00019462CE795EA0C0F06D152EA03353FF408
:107EF000FDAE1046194622E750EA410618BF52EA85
:107F000043067FF4C5AE50EA41047FF40DAF52EA58
:107F100043057FF4EBAE12E74FF0FF3C06E000BFF5
:107F20004FF0010C02E000BF4FF0010C4DF804CD02
:107F30004FEA410C7FEA6C5C4FEA430C18BF7FEAC2
:107F40006C5C1BD001B050EA410C0CBF52EA430CF0
:107F500091EA030F02BF90EA020F0020704710F170
:107F6000000F91EA030F58BF994208BF90422CBFFF
:107F7000D8176FEAE37040F0010070474FEA410CF8
:107F80007FEA6C5C02D150EA013C07D14FEA430C16
:107F90007FEA6C5CD6D152EA033CD3D05DF8040B87
:107FA000704700BF8446104662468C4619466346B9
:107FB00000E000BF01B5FFF7B7FF002848BF10F190
:107FC000000F01BD4DF808EDFFF7F4FF0CBF0120D5
:107FD00000205DF808FB00BF4DF808EDFFF7EAFF51
:107FE00034BF012000205DF808FB00BF4DF808ED0C
:107FF000FFF7E0FF94BF012000205DF808FB00BF01
:108000004DF808EDFFF7CEFF94BF012000205DF88A
:1080100008FB00BF4DF808EDFFF7C4FF34BF012097
:1080200000205DF808FB00BF4FEA410212F5001284
:1080300015D211D56FF47873B3EB625212D94FEAAF
:10804000C12343F0004343EA505311F0004F23FA99
:1080500002F018BF404270474FF00000704750EAEE
:10806000013005D111F0004008BF6FF000407047AB
:108070004FF00000704700BF4FEA4102B2F1E04309
:1080800024BFB3F5001CDCF1FE5C0DD901F0004CFF
:108090004FEAC0024CEA5070B2F1004F40EB83004F
:1080A00008BF20F00100704711F0804F21D113F17B
:1080B0003872BCBF01F00040704741F480114FEAB4
:1080C0005252C2F11802C2F1200C10FA0CF320FA3D
:1080D00002F018BF40F001004FEAC1234FEAD3235A
:1080E00003FA0CFC40EA0C0023FA02F34FEA4303C4
:1080F000CCE77FEA625307D150EA01331EBF4FF04D
:10810000FE4040F44000704701F0004040F0FE4067
:1081100040F40000704700BF4FF0FF0C1CEAD05243
:108120001EBF1CEAD15392EA0C0F93EA0C0F6FD0DA
:108130001A4480EA010C400218BF5FEA41211ED0B8
:108140004FF0006343EA501043EA5111A0FB0131A4
:108150000CF00040B1F5000F3EBF490041EAD37179
:108160005B0040EA010062F17F02FD2A1DD8B3F1F5
:10817000004F40EBC25008BF20F00100704790F064
:10818000000F0CF0004C08BF49024CEA502040EAB6
:1081900051207F3AC2BFD2F1FF0340EAC25070477C
:1081A00040F400004FF00003013A5DDC12F1190FBA
:1081B000DCBF00F000407047C2F10002410021FA2C
:1081C00002F1C2F1200200FA02FC5FEA310040F144
:1081D000000053EA4C0308BF20EADC70704792F0BD
:1081E000000F00F0004C02BF400010F4000F013AF5
:1081F000F9D040EA0C0093F0000F01F0004C02BFF0
:10820000490011F4000F013BF9D041EA0C018FE75E
:108210000CEAD15392EA0C0F18BF93EA0C0F0AD064
:1082200030F0004C18BF31F0004CD8D180EA01008A
:1082300000F00040704790F0000F17BF90F0004F23
:10824000084691F0000F91F0004F14D092EA0C0F05
:1082500001D142020FD193EA0C0F03D14B0218BF98
:10826000084608D180EA010000F0004040F0FE40DE
:1082700040F40000704740F0FE4040F4400070477A
:108280004FF0FF0C1CEAD0521EBF1CEAD15392EAF9
:108290000C0F93EA0C0F69D0A2EB030280EA010CE9
:1082A00049024FEA402037D04FF0805343EA111182
:1082B00043EA10130CF000408B4238BF5B0042F1E0
:1082C0007D024FF4000C8B4224BF5B1A40EA0C0085
:1082D000B3EB510F24BFA3EB510340EA5C00B3EBB7
:1082E000910F24BFA3EB910340EA9C00B3EBD10FA5
:1082F00024BFA3EBD10340EADC001B0118BF5FEAF7
:108300001C1CE0D1FD2A3FF650AF8B4240EBC2501F
:1083100008BF20F0010070470CF0004C4CEA5020E0
:108320007F32C2BFD2F1FF0340EAC250704740F42F
:1083300000004FF00003013A37E792F0000F00F021
:10834000004C02BF400010F4000F013AF9D040EA9F
:108350000C0093F0000F01F0004C02BF490011F433
:10836000000F013BF9D041EA0C0195E70CEAD1532B
:1083700092EA0C0F08D142027FF47DAF93EA0C0F12
:108380007FF470AF084676E793EA0C0F04D14B02F6
:108390003FF44CAF08466EE730F0004C18BF31F0A8
:1083A000004CCAD130F000427FF45CAF31F00043A2
:1083B0007FF43CAF5FE700BF4FF0FF3C06E000BF3B
:1083C0004FF0010C02E000BF4FF0010C4DF804CD5E
:1083D0004FEA40024FEA41037FEA226C18BF7FEA6E
:1083E000236C11D001B052EA530C18BF90EA010F70
:1083F00058BFB2EB030088BFC81738BF6FEAE170FF
:1084000018BF40F0010070477FEA226C02D15FEA9A
:10841000402C05D17FEA236CE4D15FEA412CE1D006
:108420005DF8040B704700BF844608466146FFE7CD
:108430000FB5FFF7C9FF002848BF10F1000F0FBDAF
:108440004DF808EDFFF7F4FF0CBF012000205DF8A8
:1084500008FB00BF4DF808EDFFF7EAFF34BF01202D
:1084600000205DF808FB00BF4DF808EDFFF7E0FFC6
:1084700094BF012000205DF808FB00BF4DF808ED17
:10848000FFF7D2FF94BF012000205DF808FB00BF7A
:108490004DF808EDFFF7C8FF34BF012000205DF85C
:1084A00008FB00BF704700BF4A1E08BF7047C0F0FE
:1084B0002481884240F21681114200F01781B0FAFF
:1084C00080F3B1FA81F2A2EB0303C3F11F0304A20C
:1084D00002EB03134FF000029F4600BFAFF3008092
:1084E000B0EBC17F00BF42EB020228BFA0EBC1701E
:1084F000B0EB817F00BF42EB020228BFA0EB81708E
:10850000B0EB417F00BF42EB020228BFA0EB4170FD
:10851000B0EB017F00BF42EB020228BFA0EB01706D
:10852000B0EBC16F00BF42EB020228BFA0EBC160FD
:10853000B0EB816F00BF42EB020228BFA0EB81606D
:10854000B0EB416F00BF42EB020228BFA0EB4160DD
:10855000B0EB016F00BF42EB020228BFA0EB01604D
:10856000B0EBC15F00BF42EB020228BFA0EBC150DD
:10857000B0EB815F00BF42EB020228BFA0EB81504D
:10858000B0EB415F00BF42EB020228BFA0EB4150BD
:10859000B0EB015F00BF42EB020228BFA0EB01502D
:1085A000B0EBC14F00BF42EB020228BFA0EBC140BD
:1085B000B0EB814F00BF42EB020228BFA0EB81402D
:1085C000B0EB414F00BF42EB020228BFA0EB41409D
:1085D000B0EB014F00BF42EB020228BFA0EB01400D
:1085E000B0EBC13F00BF42EB020228BFA0EBC1309D
:1085F000B0EB813F00BF42EB020228BFA0EB81300D
:10860000B0EB413F00BF42EB020228BFA0EB41307C
:10861000B0EB013F00BF42EB020228BFA0EB0130EC
:10862000B0EBC12F00BF42EB020228BFA0EBC1207C
:10863000B0EB812F00BF42EB020228BFA0EB8120EC
:10864000B0EB412F00BF42EB020228BFA0EB41205C
:10865000B0EB012F00BF42EB020228BFA0EB0120CC
:10866000B0EBC11F00BF42EB020228BFA0EBC1105C
:10867000B0EB811F00BF42EB020228BFA0EB8110CC
:10868000B0EB411F00BF42EB020228BFA0EB41103C
:10869000B0EB011F00BF42EB020228BFA0EB0110AC
:1086A000B0EBC10F00BF42EB020228BFA0EBC1003C
:1086B000B0EB810F00BF42EB020228BFA0EB8100AC
:1086C000B0EB410F00BF42EB020228BFA0EB41001C
:1086D000B0EB010F00BF42EB020228BFA0EB01008C
:1086E000104670470CBF012000207047B1FA81F29C
:1086F000C2F11F0220FA02F0704708B14FF0FF30BC
:10870000FFF7D0BE0029F8D02DE90340FFF7CCFEDB
:10871000BDE8064002FB00F3A1EB0301704700BF78
:1087200003460846194600F009B800BF00210A2296
:1087300001F0D2B900220A2301F02CB930B4054669
:108740000C46134602202946224630BC01F0D2B91D
:1087500049F25003C1F6FF731868704770B54AF2CA
:10876000C0764AF2C075C0F20006C0F20005761B62
:10877000B61007D0043D002455F8043F0134984753
:10878000A642F9D14AF2FC764AF2C075C0F2000660
:10879000C0F20005761B02F00DF8B61008D0043DBB
:1087A000002455F8043F01349847A642F9D170BD22
:1087B00070BD00BF49F250030146C1F6FF7318684F
:1087C00000F008B849F250030146C1F6FF7318687B
:1087D00001F052BA2DE9F04F01F10B04162C83B0D1
:1087E000074630D924F00704E30F8C422CBF19460A
:1087F00043F0010100292FD1384600F06FFCB4F599
:10880000FC7F2ED24FEAD40C49F24416C1F6FF7613
:1088100006EBCC02D368934200F01182596803F151
:108820000808DA68384621F0030499681B195C6867
:10883000CA6044F0010491605C6000F051FC404665
:1088400003B0BDE8F08F002310248C422CBF1946E2
:1088500043F001010029CFD00C234FF000083B600A
:10886000EDE75FEA542C04BF4FEAD40C4FEA4C0505
:1088700040F08F8049F24416C1F6FF7606EB85057D
:10888000EB689D4206D10DE0002A80F25581DB683D
:108890009D4207D0596821F003010A1B0F2AF3DD1E
:1088A0000CF1FF3C0CF1010C49F244123369C1F6A2
:1088B000FF7202F1080E734508BFD2F8049022D06F
:1088C000586820F00300011B0F2900F38481002960
:1088D000C2F814E0C2F810E066DAB0F5007F80F06C
:1088E0004E81C1084FF0010802EBC100891008FA5F
:1088F00001F851688568D86048EA0109C2F8049017
:108900009D60EB60836001224FEAAC0302FA03F33F
:108910004B4554D819EA030F0DD193402CF0030CAA
:1089200019EA030F0CF1040C05D15B000CF1040CE7
:1089300019EA030FF9D006EBCC09E0464846C268B5
:10894000904207D15BE1002980F28381D268904296
:1089500000F05581556825F00305291B0F29F2DD2C
:1089600090461319D56844F0010058F8084F41F0BB
:10897000010C50603846C3F804C0E560AC60736118
:108980003361C3F80CE0C3F808E0595000F0A8FBCD
:1089900055E7BCF1040F00F2DE804FEA941C0CF1A5
:1089A000380C4FEA4C0565E71A1803F108083846F9
:1089B000536843F00103536000F092FB3FE7B56852
:1089C0006B6823F0030A544504D8C4EB0A030F2B49
:1089D00000F3A4804AF69419D6F80814C1F6FF797A
:1089E00005EB0A020131D9F80030234408BF03F136
:1089F000100B06D003F580530F3323F47F6323F06D
:108A00000F0B38465946019200F05CFD019A411C5B
:108A1000804600F06881824200F23181D9F804304A
:108A200042455B44C9F8043000F06681D6F808146A
:108A300049F24410C1F6FF70013117BFC2EB0802C2
:108A4000C0F808849B18C9F8043018F007033846AA
:108A50001FBFC3F10802C3F58053904403F108021D
:108A600008EB0B0308BF4FF480521B051B0DC3EB33
:108A7000020B594600F026FD431C00F04981C8EB6B
:108A80000001594441F00101D9F80430B5424AF6D9
:108A90009412C6F808805B44C1F6FF72C8F804104F
:108AA000C9F8043018D0BAF10F0F40F20B81AAF1C7
:108AB0000C00696820F007004FF0050C05EB000E74
:108AC0000F2801F0010140EA01016960CEF804C0FD
:108AD000CEF808C000F220814AF69412D9F82C1082
:108AE000C1F6FF72B5688B42D9F8301088BFD362E7
:108AF0004AF69412C1F6FF728B4288BF13636A680C
:108B000022F003029442C4EB020301D80F2B05DCD0
:108B100038464FF0000800F0E3FA90E62A1943F0D7
:108B2000010344F0010438466C6005F10808536005
:108B3000B26000F0D5FA82E65918DA689C683846C7
:108B40004D6803F1080845F00105E26094604D604E
:108B500000F0C6FA73E6BCF1140F9CBF0CF15B0C7D
:108B60004FEA4C057FF686AEBCF1540F00F29380BD
:108B70004FEA143C0CF16E0C4FEA4C057AE6420ABF
:108B8000042A75D9142A9CBF02F15B094FEA4905F2
:108B900008D9542A00F2C9804FEA103909F16E0948
:108BA0004FEA490506EB850549F24418C1F6FF78FE
:108BB000AA68AA4279D0516821F00301884202D202
:108BC00092689542F7D1D068D6F80490D8609A6040
:108BD000D360836097E61D1941F00106556144F0AA
:108BE0000104156138465C6003F10808C5F80CE023
:108BF000C5F808E06E60695000F072FA1FE608F1EF
:108C00000108083018F0030F7FF499AE4A461CF0B3
:108C1000030FA2F108010CF1FF3C00F09E801268E6
:108C20008A42F4D072685B0093423FF6C8AE002BD4
:108C30003FF4C5AE1A4200F09580C4467BE603F1CE
:108C400008025B699A4208BF0CF1020C3FF42CAE9B
:108C5000E4E590465519D368384658F8082F6968F6
:108C6000D36041F001019A60696000F039FAE6E5ED
:108C70004FEA901909F138094FEA490592E7B542E0
:108C800049F24413C1F6FF733FF4C8AE9D686A68A9
:108C900022F0030236E7BCF5AA7F19D84FEAD43C8C
:108CA0000CF1770C4FEA4C05E4E50125D8F80410E7
:108CB0004FEAA909104605FA09F545EA0109C8F87D
:108CC000049083E701234546C8F80430002219E7E1
:108CD00040F254539C450BD84FEA944C0CF17C0C59
:108CE0004FEA4C05C6E5B5686A6822F0030209E759
:108CF000FC254FF07E0CBDE51105090D00297FF420
:108D000095AEB2680BEB0A0141F001015160E3E658
:108D100001214FF0000BB7E6384605F1080101923A
:108D200000F0AAFF019A5368D6E6B2F5AA7F06D8EA
:108D30004FEAD03909F177094FEA490532E740F2A5
:108D40005451FC258A424FF07E099EBF4FEA90495C
:108D500009F17C094FEA490524E7726822EA030217
:108D6000726060E75B0008F1040863E7032A70B4EF
:108D700022D941EA00039B0713D00578013A0C7809
:108D80000023A54206D01BE010F8015F11F8014F47
:108D9000A54215D1934203F10103F5D1002070BC27
:108DA00070470C460346043104301E682568AE4205
:108DB00008D1043A032AF4D8002ADED11046EEE79F
:108DC000281BECE721461846002AD6D1F6E700BF5B
:108DD000032A2DE9F00F09D82AB10023CC5CC45432
:108DE00001339342FAD1BDE8F00F70478307024484
:108DF0000ED0441C4D1C15F8017C04F003062346DC
:108E000001342946013504F8027C002EF3D100E03C
:108E1000034611F003046DD0D71A0D1B032F2E68E3
:108E200019DDC4F1040C4FEAC4081C1D4FEACC0C38
:108E300055F8047FC4EB0209234604310434B9F128
:108E4000030F26FA08FA07FA0CFB3E464BEA0A071C
:108E500044F8087CECDC9A42C5D901330131013277
:108E600011F8014C01330131934203F8024CF7D160
:108E7000B9E70C684033403143F8404C51F83C4C62
:108E800043F83C4C51F8384C43F8384C51F8344CCA
:108E900043F8344C51F8304C43F8304C51F82C4CDA
:108EA00043F82C4C51F8284C43F8284C51F8244CEA
:108EB00043F8244C51F8204C43F8204C51F81C4CFA
:108EC00043F81C4C51F8184C43F8184C51F8144C0A
:108ED00043F8144C51F8104C43F8104C51F80C4C1A
:108EE00043F80C4C51F8084C43F8084C51F8044C2A
:108EF00043F8044CD41A3F2CBBDC11E00C6810334F
:108F0000103143F8104C51F80C4C43F80C4C51F80C
:108F1000084C43F8084C51F8044C43F8044CD41A5C
:108F20000F2CEBDC032C96DD1C1D0D1D55F8047C6D
:108F3000161B2346294604340435032E44F8087CC6
:108F4000F4DC88E78842F0B411D98C18A0420ED224
:108F50008518531E4AB121462A4611F8014D013B9E
:108F6000B3F1FF3F02F8014DF7D1F0BC70470F2A73
:108F700047D941EA00039B0745D10C4603461546F5
:108F8000266810331034103D0F2D43F8106C54F840
:108F90000C6C43F80C6C54F8086C43F8086C54F8EB
:108FA000046C43F8046CEBD8A2F1100502F00F0436
:108FB00025F00F051035032C00EB0503294424D9B7
:108FC000A4F1040C1D460C464FEA9C0C01EB8C07E7
:108FD000043754F8046BBC4245F8046BF9D10CF12A
:108FE000010402F00302A40009191B19002ABCD0D5
:108FF00001399A1811F8014F03F8014B9342F9D146
:10900000B3E70346F2E70346F2E72246EEE700BF86
:10901000032AC9B270B408D82AB10346121803F85B
:10902000011B9342FBD170BC70478307024409D0F7
:10903000441C04F00305234604F8011C0134002DF0
:10904000F7D100E00346D51A01EB01243F2D04EBD4
:1090500004442CDD1C604033D51A43F83C4C3F2DB2
:1090600043F8384C43F8344C43F8304C43F82C4C1C
:1090700043F8284C43F8244C43F8204C43F81C4C4C
:1090800043F8184C43F8144C43F8104C43F80C4C7C
:1090900043F8084C43F8044CDCDC08E01C60103357
:1090A000D51A43F80C4C43F8084C43F8044C0F2DE8
:1090B000F4DC032D08DD1D1D561B45F8044C032E62
:1090C0002B4605F10405F7DC9A42ACD90133013295
:1090D00003F8011C01339342FAD1A4E7704700BFA3
:1090E000704700BF49F250030A46C1F6FF730146BC
:1090F000186800F001B800BF2DE9F04F0C4683B0AE
:1091000081461746002900F01C8107F10B05FFF787
:10911000E5FF54F8042C162DA4F1080A22F00306EA
:1091200075D8102100230D46BD4238BF43F001031E
:10913000002B40F00C818E426EDA49F2441B0AEBA0
:109140000600C1F6FF7BDBF808E0864500F00481ED
:10915000D0F804C02CF001088044D8F8048018F03E
:10916000010F1CBF9C4660466FD0D30700F1C3803F
:1091700054F8083CC3EB0A035A6822F00302921920
:10918000019200286CD0704500F037810CEB02088A
:10919000884565DBC1681F468068321F242A8860C5
:1091A000C16057F8080FD968C160886000F2788103
:1091B000132A9CBF394620461FD921681B2A98BF15
:1091C00004F1080099606168D96098BF03F110014B
:1091D00013D9A168242A14BF04F1100004F1180067
:1091E0001961E168596111BF03F11801226903F1A6
:1091F00020019A6104BF6269DA6102683C460A6034
:109200009A4642684A6082688A605A6805E025F09A
:1092100007052946EB0F87E7B046C5EB08030F2B80
:1092200055D80AEB080302F0010242EA0802CAF824
:1092300004205A6842F001025A6048462746FFF768
:109240004FFF384603B0BDE8F08F2CF0030C0CEB59
:109250000608884589DBC3688168CB609960DCE7D4
:10926000019A8A4247DB1F46D968321F57F8080F18
:10927000242AC160886000F2B180132A9CBF39465D
:1092800020461FD921681B2A98BF04F10800996065
:109290006168D96098BF03F1100113D9A168242A2D
:1092A00014BF04F1100004F118001961E16859615C
:1092B00011BF03F11801226903F120019A6104BF73
:1092C0006269DA6102683C46DDF8048097E70AEBE0
:1092D000050102F00102CE18154343F00103CAF85C
:1092E00004504B6048467368083143F001037360D3
:1092F00000F0C2FCA1E739464846FFF76BFA074683
:10930000D8B154F8042CA0F1080122F00103534411
:10931000994200F0BF80321F242A6AD8132A9CBFCA
:109320000346224639D8116819605168596092681D
:109330009A604846214600F09FFC4846FFF7D0FE61
:109340007FE7114603B0BDE8F04FFFF743BA0C23A7
:109350000027C9F8003074E7DEF8043005F110008A
:1093600023F0030C0CEB06038342B8BF7046FFF6F4
:10937000FCAE0AEB05025B1B43F001034846536059
:10938000274654F8043CCBF8082003F001031D43A2
:1093900044F8045CFFF7A4FE53E723681B2A98BF38
:1093A00004F1080203606368436098BF00F108039A
:1093B000B9D9A368242A14BF04F1100204F11802D9
:1093C0008360E368C36011BF00F11003216900F1FD
:1093D0001803016104BF61694161A4E72146384671
:1093E0000093FFF7AFFD9DE808013C469A465A6896
:1093F00013E72146FFF7A6FD9BE7019805F1100250
:109400000CEB00089045FFF62BAF1F46D968321FC2
:1094100057F8080F242AC16088604BD8132A9CBFD4
:109420003A4621461FD921681B2A98BF03F1100232
:1094300099606168D96098BF04F1080113D9A168E7
:10944000242A14BF03F1180203F120021961E16814
:10945000596111BF04F11001206904F118019861EC
:1094600004BF6069D8610868106048685060896806
:1094700091605A19C5EB080141F00101484651605D
:109480005968CBF8082001F001010D435D60FFF73A
:1094900027FED6E650F8043C23F00308B044BCE6AF
:1094A000214638460093FFF74DFD009B3C469A4607
:1094B0005A68B2E6384621460093FFF743FD009B09
:1094C000D7E700BF38B54AF6D814C1F6FF74054691
:1094D000084600232360FAF76BFC431C00D038BD1C
:1094E0002368002BFBD02B6038BD00BFC9B2F0B49D
:1094F00000294BD083070FD00378002B73D09942FB
:1095000042D0431C05E013F8012B002A3BD09142C6
:109510003AD09A071846F6D1036841EA0127A3F129
:10952000013247EA074722EA030212F0803F1CD1CA
:109530007B40A3F1013222EA030313F0803F14D1F0
:10954000021D02E014F0803F0FD1104652F8043B98
:10955000A3F1013687EA030426EA0303A4F10135E7
:1095600013F0803F25EA0404ECD00378002B3AD0B6
:10957000994209D0431C01E0914205D0184613F8E6
:10958000012B002AF8D11046F0BC704781070DD09E
:109590000378002BF8D0431C02E00278002AF3D0B5
:1095A00013F0030F184603F10103F6D10368A3F18A
:1095B000013222EA030313F0803F0AD1021D104654
:1095C00052F8041BA1F1013424EA010111F0803F9B
:1095D000F5D00378002BD7D0431C1846013302780E
:1095E000002AFAD1D0E71846CEE700BF80EA010290
:1095F00012F0030F40F03A8010F0030220F0030055
:1096000021F0030150F804CB08BF51F8043B0DD002
:1096100082F003024FEAC2026FF07F4323FA02F2A4
:1096200051F8043B4CEA020C43EA0203ACF101326C
:109630009C4501BF22EA0C0212F0803F50F804CB97
:1096400051F8043BF2D04FEA0C604FEA1C2C012881
:1096500028BFB0EB036F08BF1B0AF4D003F0FF0371
:109660004FEA1060A0EB0300704700BF10F0030F3B
:109670000AD010F8012B11F8013B012A28BF9A42A9
:10968000F4D0A2EB030070474DF8045D4DF8044D93
:109690004FF0010242EA022242EA024201F0030CC8
:1096A00021F0030150F8044B51F8045BBCF1020FA8
:1096B00026D04BD824F07F4CBCEB152FA4EB020333
:1096C00023EA04030DD113EAC21308BF51F8045B67
:1096D0000AD18CEA040CBCEB056F0CD150F8044B9A
:1096E000E8E74FEA15255CE033F07F4352D10D786F
:1096F0004FEA146C55E04FEA146C05F0FF0550E09A
:109700004FEA044CA4EB02034FEA1C4C23EA040387
:10971000BCEB154F17D113EAC21308BF51F8045B15
:1097200007D18CEA040CBCEB054F08D150F8044B70
:10973000E6E71B042ED10D884FEA144C31E04FEAC6
:1097400005454FEA144C4FEA15452AE004F0FF0C9A
:10975000BCEB156FA4EB020323EA04030DD113EA5B
:10976000C21308BF51F8045B0AD18CEA040CBCEBAD
:10977000052F0AD150F8044BE8E74FEA156510E0D1
:1097800014F0FF0F06D051F8045B4FEA142C25F0BB
:109790007F4506E04FF000005DF8044B5DF8045B88
:1097A00070470CF0FF0205F0FF00012828BF90422F
:1097B00004BF4FEA1C2C2D0AF3D0A2EB00005DF889
:1097C000044B5DF8045B704780EA0102844612F0A6
:1097D000030F4FD111F0030F32D14DF8044D11F0AA
:1097E000040F51F8043B0BD0A3F101329A4312F05D
:1097F000803F04BF4CF8043B51F8043B16D100BF36
:1098000051F8044BA3F101329A4312F0803FA4F1C6
:1098100001320BD14CF8043BA24312F0803F04BF4D
:1098200051F8043B4CF8044BEAD023460CF8013BBA
:1098300013F0FF0F4FEA3323F8D15DF8044B704764
:1098400011F0010F06D011F8012B0CF8012B002AA2
:1098500008BF704711F0020FBFD031F8022B12F091
:10986000FF0F16BF2CF8022B8CF8002012F47F4F4C
:10987000B3D1704711F8012B0CF8012B002AF9D154
:10988000704700BF70B4002A45D041EA000313F0CE
:10989000030329D1032A27D905680C68A54223D1DF
:1098A000141F3AD0A5F1013222EA050515F0803FD8
:1098B0000DD03AE05B686A68A3F10135934225EA6E
:1098C00003052ED1043C28D015F0803F27D10D464A
:1098D000034604310430032CECD8661E2CB91C79E5
:1098E0002A79A01A70BC7047561E04780A789442F0
:1098F000F7D1C6B18CB101368B1C891904E08B42BB
:1099000003F101030BD044B113F8012C10F8014FFF
:109910009442F4D0E5E71046E4E72046E2E7002071
:10992000E0E7661EE1E73046DCE71846DAE700BF0D
:1099300041EA000313F0030F034670B425D0AAB127
:109940000C78013A03F8014B4CB11C4672B111F886
:10995000015F013A04F8015B2346002DF6D12AB1DC
:109960009A18002103F8011B9342FBD170BC704789
:109970000E4651F8044BA4F1013525EA040515F013
:10998000803F05D1043A43F8044B032AF0D8D6E7C8
:109990003146D4E72DE9F04F49F25454C1F6FF7433
:1099A00085B099460B46D4F80080029103901C467E
:1099B00014F8015B08EB05012346497801F0080122
:1099C000C9B20029F3D12D2D7BD02B2D05BF244604
:1099D0000B460B4614F8015B39F0100112D1D9F196
:1099E000010038BF0020302D04D058B14FF00A09D3
:1099F000CB4608E0217801F0DF01582965D008B195
:109A00004FF00809CB46002B59460CBF6FF00046BB
:109A10004FF000468DE80C0030460027FEF772FE3E
:109A200030468A465946FEF73FFDBC469DE80C008D
:109A300016E0303DA94525DD844594BF0021012174
:109A400051EAD77729D15545D4BF0021012184455A
:109A500018BF002109BB0BFB0C5C012714F8015B4C
:109A600008EB0501497801F00406F6B2002EE0D1BA
:109A700011F0030106D0012914BF572137216D1AB7
:109A8000A945D9DC791C0BD0C3B9604612B197B98E
:109A9000029B136005B0BDE8F08F4FF0FF37DDE7A4
:109AA0000399002B0CBF6FF000404FF000402223C1
:109AB0000B60002AEED0013C0294E9E7CCF1000CE7
:109AC000E3E714F8015B012386E74FF0100965789E
:109AD000CB46023497E700BF30B449F25004C1F6D8
:109AE000FF740D46134601462A46206830BCFFF736
:109AF00051BF00BF2DE9F0414AF24864C0F20004B2
:109B000084B007462568AC6C002C42D066681F2ED6
:109B10001ADD48F2B574C0F2000424B94FF0FF30EA
:109B200004B0BDE8F0818C20039102920193FEF70E
:109B300041FE0399029A019B04460028EED0A86CCE
:109B4000002684E84100AC64DFB1D4F8886026B315
:109B5000D6F8008165680120022F05F1200C00FA7B
:109B600005F046F8252048EA000246F82C3008BFE8
:109B7000D6F80431C6F8002104BF1843C6F8040122
:109B800000E06568AB1C00200135656044F82310D7
:109B9000C6E705F14C04AC64B8E748F2B570C0F212
:109BA00000000028BAD04FF4847003910292019310
:109BB000FEF700FE0399029A019B06460028ADD0ED
:109BC0000020C6F80001C6F804018046C4F8886089
:109BD000C0E700BFF8B549F24414C1F6FF740F4660
:109BE0000546FFF77BFAA3685E6826F0030606F6D3
:109BF000EF73DF1B3F0B013F3F03B7F5805F07DBD0
:109C000000212846FFF75EFCA3689B19984204D008
:109C10002846FFF765FA0020F8BD79422846FFF78D
:109C200051FC013010D04AF69813A168C1F6FF73B9
:109C3000F61B284646F001061A684E60D71B1F60C7
:109C4000FFF74EFA0120F8BD00212846FFF73AFC45
:109C5000A368C21A0F2ADBDD49F24C544AF6981168
:109C6000C1F6FF74C1F6FF7142F001025A60236829
:109C7000C01A0860CCE700BF2DE9F0410E468046CF
:109C800000295CD0FFF72AFA49F2441556F8041C63
:109C9000C1F6FF75A6F1080421F00103AF68E218D0
:109CA0009742506820F0030067D011F00101506026
:109CB00035D000211618766816F0010F06D11B1852
:109CC000906800294DD0D268C260906043F00102D4
:109CD000E3506260F1B9B3F5007F32D35A0A042A27
:109CE0006CD898093830410005EB810549F24411E0
:109CF000C1F6FF71AA68AA426BD0516821F0030136
:109D00008B4202D292689542F7D1D368E360A26099
:109D1000D4609C604046BDE8F041FFF7E1B956F8D9
:109D2000086C05F1080CA41B9B19A668664543D076
:109D3000D4F80CC0C6F80CC0CCF80860BAE7BDE88F
:109D4000F081DB080121686805EBC3029B1001FA72
:109D500003F3E260916818436860A160CC6094608E
:109D6000D8E7294EB042AED16C6143F001022C61BC
:109D7000E060A0606260E350CCE7C018CB0707D476
:109D800056F8083CE41AC018A268E368D3609A60E9
:109D900049F2505240F00103C1F6FF726360AC60BB
:109DA00013689842B6D34AF694134046C1F6FF733F
:109DB0001968FFF70FFFADE701217BE702F15B00B8
:109DC0004100142A90D9542A0CD8180B6E30410047
:109DD0008AE701264D688010134606FA00F0054315
:109DE0004D6093E7B2F5AA7F03D8D80B77304100D6
:109DF0007AE740F254518A4203D8980C7C304100F3
:109E000072E7FC217E206FE74C91FF1FFFFFFFFFF1
:109E10000000000000000000C13D00000000000044
:109E20000100000002000000040000000800000023
:109E30001000000020000000400000008000000032
:109E400000010000030000000600000009000000FF
:109E50000C0000002F0030006469726563746F723B
:109E600079206E6F7420666F756E64005F007C00F1
:109E700042616E6B3A00204368616E6E656C3A0019
:109E80002046696C653A004D5554453D00444543B4
:109E90004C49434B3D0053686F774D657465723D87
:109EA000006D65746572484944453D004368616EC4
:109EB000506F74496D6D6564696174653D004368F8
:109EC000616E4356496D6D6564696174653D00530B
:109ED00074617274506F74496D6D65646961746505
:109EE0003D0053746172744356496D6D65646961D8
:109EF00074653D004D555445004445434C49434B22
:109F00000053686F774D65746572006D6574657296
:109F100048494445004368616E506F74496D6D65F2
:109F20006469617465004368616E4356496D6D658F
:109F30006469617465005374617274506F74496D23
:109F40006D65646961746500537461727443564948
:109F50006D6D656469617465005374617274435614
:109F600044697669646572004C6F6F70696E670052
:109F70006572726F72206F70656E696E67207365AF
:109F80007474696E67732E7478740053746172749C
:109F90004356446976696465723D004C6F6F706921
:109FA0006E673D002062616E6B7320666F756E6434
:109FB000004F70656E2062616E6B002066696C6593
:109FC0007320666F756E6420696E2062616E6B200F
:109FD00000537769746368696E6720746F206261EB
:109FE0006E6B20004E4F2046494C4553204552523F
:109FF0004F5200617474656D7074696E6720746F80
:10A0000020706C61792066696C6520006F72206D2C
:10A010006179626520005241570000000100040090
:10A020000B0013001E002C003C004E0063007B0060
:10A030009500B100D000F10014013A0163018E01D6
:10A04000BB01EA011D0251028802C102FC023A036F
:10A050007B03BD03020449049304DF042D057D0541
:10A06000D00524067C06D50630078E07EE0750087B
:10A07000B4081A098309ED095A0AC90A390BAC0B4D
:10A08000210C980C100D8B0D080E860E070F890FF2
:10A090000D1093101B11A5113112BE124D13DE13BA
:10A0A000701404159A153216CB16651701189F18EF
:10A0B0003E19DF19811A251BCA1B711C181DC21DF0
:10A0C0006C1E181FC51F73202321D421862239231B
:10A0D000ED23A22458250F26C82681273B28F628E1
:10A0E000B2296F2A2D2BEC2BAB2C6B2D2C2EED2EA9
:10A0F000AF2F72303531F931BD32823348340E35ED
:10A10000D4359B3662372938F138B939813A493B21
:10A11000123CDB3CA43D6D3E363FFF3FC8409141C1
:10A120005A422343EB43B4447C4545460C47D4474D
:10A130009C486349294AF04AB64B7B4C404D044E3B
:10A14000C84E8C4F4E501051D2519352535312540B
:10A15000D0548E554B560757C2577C583659EE5936
:10A16000A55A5C5B115CC55C785D2A5EDB5E8A5F2C
:10A170003960E66091613C62E5628D633364D96465
:10A180007C651E66BF665F67FC6798683369CC694B
:10A19000646AF96A8E6B206CB16C406DCD6D596E3E
:10A1A000E26E6A6FF06F7570F7707871F6717372A6
:10A1B000EE726673DD735274C5743675A4751176CC
:10A1C0007B76E4764A77AE7710787078CE78297906
:10A1D0008379DA792F7A817AD27A207B6C7BB57B8E
:10A1E000FC7B417C847CC47C027D3E7D777DAE7DA2
:10A1F000E27D147E447E717E9C7EC47EEA7E0E7F6C
:10A200002F7F4E7F6A7F847F9B7FB07FC37FD37F0A
:10A21000E17FEC7FF47FFB7FFE7FFF7FFFFFFFFF8F
:10A220000000000000000000051700000000000012
:10A2300000000000000000004517000000000000C2
:10A240000000000000000000611900000000000094
:10A250000000000000000000511B00000000000092
:10A260006E203D0002000300040005000600080007
:10A270000A000C001000140018002000280038000C
:10A28000400060008000C0000001800100028002E8
:10A290000003FFFF000000800000018000000000BC
:10A2A0000000028000000100011000000000020018
:10A2B0000110010003200000010002000320010042
:10A2C00004300000032002000320030005400000CA
:10A2D0000540010006500000065001000760000024
:10A2E00007600100087000000760020008700100AC
:10A2F0000000000000000000391E0000571E000092
:10A30000911F00009B1E0000AD1E00004D1E0000AE
:10A310007C3C3E5E2B3D3F2F5B5D3B2C2A225C004C
:10A3200000000000000000005533000085510000CF
:10A330000000000000000000653700000138000048
:10A34000A1370000B5370000DD3700009D37000061
:10A35000050E08090D0C06070F04001303931A924B
:10A3600017C585848687C4FF6FF07F030370037869
:10A3700013F0800FFBD070474008FE4340A004401C
:10A380004408FE4344A004400018FE4300C00440BB
:10A390003000FE43309004403400FE4334900440CB
:10A3A0001C18FE431CC004401018FE4310C004409B
:10A3B0000818FE4308C004400C18FE430CC00440BB
:10A3C0000C10FE430CB004401010FE4310B00440CB
:10A3D0001810FE4318B004401C10FE431CB004408B
:10A3E0001410FE4314B004400418FE4304C004409B
:10A3F0000010FE4300B004400008FE4300A00440EB
:10A400000408FE4304A004400C08FE430CA00440D2
:10A410000808FE4308A004401418FE4314C004407A
:10A420001818FE4318C004400410FE4304B0044052
:10A430000810FE4308B004401400FE43149004408A
:10A440004C08FE434CA004400420FE4304D00440CA
:10A450002410FE4324B004402010FE4320B00440EA
:10A460002810FE4328B004402C10FE432CB00440BA
:10A470000020FE4300D004404808FE4348A00440AA
:10A480001000FE43109004400D0AFFFFFFFFFFFF86
:10A4900000000000000000004F5200004752000082
:10A4A000615200005D5200005952000055520000F8
:10A4B0000015191500010000B08FFF1F12000000E9
:10A4C00000020000DA8FFF1F4300000000030000BD
:10A4D0003490FF1F0000000001030904C28FFF1F1A
:10A4E00000000000020309041E90FF1F000000008E
:10A4F000030309043890FF1F000000000000000063
:10A50000000000000000000000000000000000004B
:10A5100051620000756200009962000091620000C3
:10A52000956200008D620000A7620000B962000021
:10A53000A36200009D620000896200008562000045
:10A5400015620000216200002D62000039620000E7
:10A550005D62000045620000000000000000000095
:10A5600035630000596300007D63000075630000DF
:10A5700079630000716300008B6300009D6300003D
:10A5800087630000816300006D6300006963000061
:10A59000F962000005630000116300001D63000004
:10A5A000416300002963000000000000000000007B
:10A5B000196400003D6400006164000059640000FB
:10A5C0005D640000556400006F6400008164000059
:10A5D0006B64000065640000516400004D6400007D
:10A5E000DD630000E9630000F56300000164000022
:10A5F000256400000D640000706F7700FFFFFFFF0F
:10A60000000000000000F03F000000000000F83FE4
:10A61000000000000000000006D0CF43EBFD4C3EE0
:10A6200000000000000000000000004003B8E23F0E
:10A6300000FFFFFFFFFFFFFF0000000000003043AE
:10A6400000000000000030C35490FF1F43000000D2
:10A6500000202020202020202020282828282820F2
:10A6600020202020202020202020202020202020EA
:10A670002088101010101010101010101010101052
:10A680001004040404040404040404101010101042
:10A69000101041414141414101010101010101010C
:10A6A000010101010101010101010101101010105E
:10A6B00010104242424242420202020202020202DE
:10A6C0000202020202020202020202021010101032
:10A6D000200000000000000000000000000000005A
:10A6E000000000000000000000000000000000006A
:10A6F000000000000000000000000000000000005A
:10A700000000000000000000000000000000000049
:10A710000000000000000000000000000000000039
:10A720000000000000000000000000000000000029
:10A730000000000000000000000000000000000019
:10A740000000000000000000000000000000000009
:10A7500000000000000000000000000000000000F9
:10A7600000000000000000000000000000000000E9
:10A7700000000000000000000000000000000000D9
:10A7800000000000000000000000000000000000C9
:10A7900000000000000000000000000000000000B9
:10A7A00000000000000000000000000000000000A9
:10A7B00000000000F8B500BFF8BC08BC9E4670471A
:10A7C00099040000691400005F160000A918000039
:10A7D000C1180000091B0000211B0000391B0000EC
:10A7E00095230000F12A0000D139000069520000D1
:0CA7F000DD620000C1630000A5640000F1
:10A7FC000000000001000000FA000000D00700007B
:10A80C000F00000028000000010000000A000000FA
:10A81C000600000001000000020000000100000022
:10A82C000300000001000000F40100000A00000019
:10A83C00FFFFFFFF0A040000DCA9FF1FFFFFFFFF63
:10A84C001201000202000040C01683040001010244
:10A85C00030118035400650065006E007300790055
:10A86C006400750069006E006F000902430002016C
:10A87C0000C032090400000102020100052400108E
:10A88C000105240101010424020605240600010728
:10A89C0005820310004009040100020A00000007B1
:10A8AC000503024000000705840240000000160367
:10A8BC0055005300420020005300650072006900EF
:10A8CC0061006C00040309040C030000000000008C
:10A8DC00000000000000000000000000000001006B
:10A8EC005490FF1F0000000094A7000074A7000004
:10A8FC0054A7000000000000000000000000000051
:10A90C00000000004CA60000000000000000000049
:10A91C00000000000000000000000000000000002B
:10A92C00000000000000000000000000000000001B
:10A93C00000000000000000000000000000000000B
:10A94C0000000000000000000000000000000000FB
:10A95C0000000000000000000000000000000000EB
:10A96C0000000000000000000000000000000000DB
:10A97C0000000000000000000000000000000000CB
:10A98C0000000000000000000000000000000000BB
:10A99C0000000000000000000000000000000000AB
:10A9AC00000000000000000000000000000000009B
:10A9BC00000000000000000000000000000000008B
:10A9CC00000000000000000000000000000000007B
:10A9DC000000000000000000000000004491FF1F78
:10A9EC004491FF1F4C91FF1F4C91FF1F5491FF1F6F
:10A9FC005491FF1F5C91FF1F5C91FF1F6491FF1F1F
:10AA0C006491FF1F6C91FF1F6C91FF1F7491FF1FCE
:10AA1C007491FF1F7C91FF1F7C91FF1F8491FF1F7E
:10AA2C008491FF1F8C91FF1F8C91FF1F9491FF1F2E
:10AA3C009491FF1F9C91FF1F9C91FF1FA491FF1FDE
:10AA4C00A491FF1FAC91FF1FAC91FF1FB491FF1F8E
:10AA5C00B491FF1FBC91FF1FBC91FF1FC491FF1F3E
:10AA6C00C491FF1FCC91FF1FCC91FF1FD491FF1FEE
:10AA7C00D491FF1FDC91FF1FDC91FF1FE491FF1F9E
:10AA8C00E491FF1FEC91FF1FEC91FF1FF491FF1F4E
:10AA9C00F491FF1FFC91FF1FFC91FF1F0492FF1FFD
:10AAAC000492FF1F0C92FF1F0C92FF1F1492FF1FAA
:10AABC001492FF1F1C92FF1F1C92FF1F2492FF1F5A
:10AACC002492FF1F2C92FF1F2C92FF1F3492FF1F0A
:10AADC003492FF1F3C92FF1F3C92FF1F4492FF1FBA
:10AAEC004492FF1F4C92FF1F4C92FF1F5492FF1F6A
:10AAFC005492FF1F5C92FF1F5C92FF1F6492FF1F1A
:10AB0C006492FF1F6C92FF1F6C92FF1F7492FF1FC9
:10AB1C007492FF1F7C92FF1F7C92FF1F8492FF1F79
:10AB2C008492FF1F8C92FF1F8C92FF1F9492FF1F29
:10AB3C009492FF1F9C92FF1F9C92FF1FA492FF1FD9
:10AB4C00A492FF1FAC92FF1FAC92FF1FB492FF1F89
:10AB5C00B492FF1FBC92FF1FBC92FF1FC492FF1F39
:10AB6C00C492FF1FCC92FF1FCC92FF1FD492FF1FE9
:10AB7C00D492FF1FDC92FF1FDC92FF1FE492FF1F99
:10AB8C00E492FF1FEC92FF1FEC92FF1FF492FF1F49
:10AB9C00F492FF1FFC92FF1FFC92FF1F0493FF1FF8
:10ABAC000493FF1F0C93FF1F0C93FF1F1493FF1FA5
:10ABBC001493FF1F1C93FF1F1C93FF1F2493FF1F55
:10ABCC002493FF1F2C93FF1F2C93FF1F3493FF1F05
:10ABDC003493FF1F3C93FF1F3C93FF1F4493FF1FB5
:10ABEC004493FF1F4C93FF1F4C93FF1F5493FF1F65
:10ABFC005493FF1F5C93FF1F5C93FF1F6493FF1F15
:10AC0C006493FF1F6C93FF1F6C93FF1F7493FF1FC4
:10AC1C007493FF1F7C93FF1F7C93FF1F8493FF1F74
:10AC2C008493FF1F8C93FF1F8C93FF1F9493FF1F24
:10AC3C009493FF1F9C93FF1F9C93FF1FA493FF1FD4
:10AC4C00A493FF1FAC93FF1FAC93FF1FB493FF1F84
:10AC5C00B493FF1FBC93FF1FBC93FF1FC493FF1F34
:10AC6C00C493FF1FCC93FF1FCC93FF1FD493FF1FE4
:10AC7C00D493FF1FDC93FF1FDC93FF1FE493FF1F94
:10AC8C00E493FF1FEC93FF1FEC93FF1FF493FF1F44
:10AC9C00F493FF1FFC93FF1FFC93FF1F0494FF1FF3
:10ACAC000494FF1F0C94FF1F0C94FF1F1494FF1FA0
:10ACBC001494FF1F1C94FF1F1C94FF1F2494FF1F50
:10ACCC002494FF1F2C94FF1F2C94FF1F3494FF1F00
:10ACDC003494FF1F3C94FF1F3C94FF1F4494FF1FB0
:10ACEC004494FF1F4C94FF1F4C94FF1F5494FF1F60
:10ACFC005494FF1F5C94FF1F5C94FF1F6494FF1F10
:10AD0C006494FF1F6C94FF1F6C94FF1F7494FF1FBF
:10AD1C007494FF1F7C94FF1F7C94FF1F8494FF1F6F
:10AD2C008494FF1F8C94FF1F8C94FF1F9494FF1F1F
:10AD3C009494FF1F9C94FF1F9C94FF1FA494FF1FCF
:10AD4C00A494FF1FAC94FF1FAC94FF1FB494FF1F7F
:10AD5C00B494FF1FBC94FF1FBC94FF1FC494FF1F2F
:10AD6C00C494FF1FCC94FF1FCC94FF1FD494FF1FDF
:10AD7C00D494FF1FDC94FF1FDC94FF1FE494FF1F8F
:10AD8C00E494FF1FEC94FF1FEC94FF1FF494FF1F3F
:10AD9C00F494FF1FFC94FF1FFC94FF1F0495FF1FEE
:10ADAC000495FF1F0C95FF1F0C95FF1F1495FF1F9B
:10ADBC001495FF1F1C95FF1F1C95FF1F2495FF1F4B
:10ADCC002495FF1F2C95FF1F2C95FF1F3495FF1FFB
:10ADDC003495FF1F3C95FF1F3C95FF1FFFFFFFFFA6
:08ADEC000000020050A6000067
:00000001FF
